:100000000C94C90D0C94F10D0C94F10D0C94F10DA0
:100010000C94F10D0C94F10D0C94F10D0C94F10D68
:100020000C94F10D0C94F10D0C941C1B0C948B1B77
:100030000C94F10D0C94F10D0C94F10D0C94F10D48
:100040000C94F10D0C94F01E0C94F10D0C94F10D28
:100050000C94F10D0C94F10D0C94F10D0C94BD1D4C
:100060000C94F10D0C94F10D0C94F10D0C94F10D18
:100070000C94F10D0C94F10D0C94F10D0C94F10D08
:100080000C94071E0C94F10D0C94F10D0C94F10DD1
:100090000C94F10D0C94F10D0C94F10D0C94F10DE8
:1000A0000C94F10D0C94F10D0C94F10D0608087EE2
:1000B0007E7E7E08FFFFFFFFFF080E76767676785D
:1000C0007E7676767608F8F7F7F7F708787676761C
:1000D000760E08767676760EFEFEFEFEFE08087632
:1000E0007676760878767676760810107DF3FDF9C8
:1000F0007A0C00000000000000000000000000007A
:100100000000000000000000000000000080C0406F
:10011000C600FF000000000000000000040F142EC5
:100120003F3E1C000000000000000000FFFF3F7F7A
:10013000362C540C58F0FEFFDCB8F00302060AFA25
:10014000FAFAFBFC9FDDF0914BC6000000000001B5
:100150000303070B0B07090C0720505E81E3FEE049
:10016000C0A0B0D0B010B0E0408000020503830012
:100170000000C041478D38E95454555920FEFC3FDA
:10018000FC3C9810E0000003040813111F0F0E0838
:10019000081C3F3F5F2E423D000100386844FC1AB6
:1001A000CECB9DCBCDD13FC6C4F8F8980888B040DF
:1001B000000070882B1EFA6242424AF9FFFFE1F00C
:1001C00010E100000000000000010100000000003C
:1001D00000010101020201000000C0FF1050F8B44C
:1001E0008EDBADABA5C316E4F8D028FFF070F01F8E
:1001F000020303F6F9F2E242C24241FBFF7BF1FF48
:10020000800003000004040003040404030000034E
:1002100004040407010080404080601C3A958983F3
:10022000CF1AF2FCF07088488870030409080F0F99
:100230001DA5C5858482477F3C7E5C621E00000050
:100240000000000006030303030600000000000096
:1002500000006C5B417AFC44EE0391DDCBCD9A8CBF
:10026000B0E00000003C4498FC7F644041E2F2FEB4
:10027000EE060F131B13160C000000000000000711
:10028000050505060000000000000080601CBA950E
:1002900049C34F9A32FCF8C46438000000011F279C
:1002A000C5CDB5858546737F7C9C48241800000029
:1002B000000C0B0B0B0B0F000000000000007F8BED
:1002C0000FFFD7E7FE16C3A5ABADDB8EB9E151F149
:1002D000BFC100000107FB03F7FDFAE2C242C2E121
:1002E0007E3F9BFFD9B000000000010307070F0B02
:1002F00009040300010100000103302E213F7C7836
:10030000C4C61F030D8BDDCA9CF0F87F312E300070
:1003100000E030501079FFE1C28282E2511D13E10A
:1003200000000000000000010202020100000000C5
:10033000010202020100000000F8160F854B45CBB8
:10034000C6ECF0ECE4FF38000000031E7EFEFFE385
:10035000F3F3FF6C2FBEBC5C18000000000001012D
:10036000010100010101000000F8B48E9BCDCBC556
:100370008316E4782C5448B800C06013FEDE9E9EBD
:100380009FB7FFF4D40AF900010203010100000045
:10039000000001010100102F2162FEF8E41E8B8D88
:1003A0009B8D8B1EE4E4F8FE62212F10008040201C
:1003B00060B177FFF9E28282E1F1FFF3F0600000C3
:1003C000000000010206040406030100000003020D
:1003D00002040405030000000038544ADDCBCDC3FD
:1003E0004F16E4782C7FC8B8E0103019FAFECE8E94
:1003F0008687C7FFF4E41FF100010202010000003C
:10040000000000010302010000000000D8649C4AC3
:1004100055C9830F1AF2FCF0F87484C458201028D0
:1004200024244E3F0FDDE5E5C5050281707F3C4E7B
:10043000221C0000000000000000000D0B0B0B0F41
:100440000100000000000000000000000098E41C13
:100450000A158943CF1AF2FCF87C3C423216181078
:100460002C242F4E3EDDE5E5C50482F1F87F3CB833
:10047000C00000000000000000000D0B0B0B0F017E
:100480000001010100000000001826217A7AFCF228
:100490001A8F43C9558A9E74D880000000001C3210
:1004A00042467FF9828485C5E5FDC78F1110190B7F
:1004B00004000000000000000000060B0B0B0B0DF9
:1004C000000000000000000000D8649C4A55C98369
:1004D0000F1AF2FCF0F87484C45820102824244E1B
:1004E0003F0FDDE5E5C5050281707F3C4E221C0013
:1004F00000000000000000000D0B0B0B0F010000BE
:10050000000000000000003629217A7AFCF21A8FE0
:10051000C3C9E7A5AB46DCA08000001C3242467F81
:10052000F9828485C5E5FDC78F1510090700000015
:10053000000000000000060B0B0B0B0D000000007C
:100540000000000000000000C0E0F0787C78FC783B
:100550007870F0E0C0000000000000000000000023
:100560000000000000000000C0F0F8FCFE31151F84
:10057000003E11152615113E001F1531FEFCF8F046
:10058000C0000000000000000000000000003FFF6D
:10059000FF7F3F1C1060A040848282828440A06064
:1005A000901C3F7FFFFF3F00F800000000000000AC
:1005B000000000008098FF7C787A7CFDEBFAE5C0B3
:1005C000C0C0E5FAEBFD7C7A787CFF988000FFFCE8
:1005D000FCFCCC0404CCFCFC00030404040407056C
:1005E0000404050503010111131D151414151F142E
:1005F0001414141B0F03030302020202030300007E
:10060000000000000000C0E0F0787878F87878709A
:10061000F0E0C0000000000000000000000000004A
:10062000000000000000C0F0F8FCFE31151F003E85
:1006300011152615113E001F1531FEFCF8F0C00003
:1006400000000000000000000000F8003FFFFF7FF6
:100650003F1C1060A040848282828440A060901C75
:100660003F7FFFFF3F00F800000000000000000097
:10067000FF008098FF7C787A7CFDEBFAE5C0C0C073
:10068000E5FAEBFD7C7A787CFF988000FFFCFCFCAF
:10069000CC0404CCFCFC0F1B141414141F151414EC
:1006A000151D13110111131D151414151F14141405
:1006B000141B0F030303020202020303FE030101E2
:1006C0000101FF01C1E1F17F7D79FC787870F0E0F4
:1006D000C00000000000000000000000000000005A
:1006E0000000FF00C0F0F8FCFF31151F003E11159F
:1006F0002615113E001F1531FEFCF8F0C000000069
:100700000000000000000000F9003FFFFF7F3F1CD9
:100710001060A040848282828440A060901C3F7F51
:10072000FFFF3F00F8000000000000000000FF0095
:100730008098FF7C787A7CFDEBFAE5C0C0C0E5FAD2
:10074000EBFD7C7A787CFF988000FFFCFCFCCC04FD
:1007500004CCFCFC0F1B141414141F151414151DC9
:1007600013110111131D151414151F141414141B47
:100770000F030303020202020303FE03010101014E
:10078000FF01C1E1F17F7D79FC79797FF1E1C10160
:10079000FF0101010103FE00000000000000000055
:1007A000FF00C0F0F8FCFF31151F003E11152615A3
:1007B000113E001F1531FFFCF8F0C000FF000000E3
:1007C000000000000000F9003FFFFF7F3F1C1060A9
:1007D000A040848282828440A060901C3F7FFFFF03
:1007E0003F00F9000000000000000000FF008098BA
:1007F000FF7C787A7CFDEBFAE5C0C0C0E5FAEBFD42
:100800007C7A787CFF988000FFFCFCFCCC0404CC54
:10081000FCFC0F1B141414141F151414151D1311B4
:100820000111131D151414151F141414141B0F0398
:100830000303020202020303C060129D1283171F0A
:100840001F2644F8010303040508090A08040603E7
:100850001F02021F001F00121509001215091010B7
:100860000408081C3E266C66C2E781C30000000035
:100870000000000000000000000000000000000078
:1008800010103C3C32161A113B313B0000000000B6
:100890000000000000000000000000000000000058
:1008A0000060E090BCDF97C280C000000000000044
:1008B0000101000101000101010100000000000030
:1008C00078CFACBC70C00000000000000000000049
:1008D00000070F0A010507000000000000000000EB
:1008E00000000080803F00F80000000000000000D1
:1008F000E0C0E1CB6FDEC871B080000000000000F6
:100900003B313B111A16323C3C1010000000000035
:1009100000000000000000000000000000000000D7
:10092000C080C297DFBC90E06000000000000000C3
:1009300001010101000101000101000000000000AF
:100940001010A070E0D4399E0C00000000000000E0
:10095000000000000101070A171C00000000000051
:1009600000000A0C5FFC383068585020000000007E
:100970000000000507030000000000000000000068
:1009800000008095DEFC60D0B0A0400000000000B8
:100990000000000103000000000000000000000053
:1009A0000000050E56F77F060D0B0A04000000003C
:1009B0000000000001000000000000000000000036
:1009C000000028183C5CF8EE8D0B0A0400000000C3
:1009D0000000000000010507030000000000000007
:1009E000000000000000240027002A002D00300035
:1009F00000000000250028002B002E003100040814
:100A00000201104080401020408040800802040114
:100A10008040201002011080102040402004040477
:100A20000404030405020202020403020202020695
:100A30000606060606040402020204040601150165
:100A4000260137014A015D01720188019F01B80149
:100A5000D201EE010B022A024B026E029302BA028D
:100A6000E40210033F037003A403DC0317045504DE
:100A70009704DD0427057505C80520067D06E006F8
:100A80004907B8072D08A9082D09B9094D0AEA0A2E
:100A9000900B400CFA0CC00D910E6F0F5A105311B1
:100AA0005B1272139A14D41520178018F519801B45
:100AB000231DDE1EB420A622B524E4263429A72B4C
:100AC000402E0031EA330037453ABC3D68414C4581
:100AD0006B49C84D68524F57805C00621011121369
:100AE000151617181A1C1D1F21232527292C2E31F6
:100AF00034373A3E4145494E52575C62686E757BC9
:100B0000838B939CA5AFB9C4D0DCE9F7D5F08D14E5
:100B1000A1C881CFD9F1AF20002808E0F9E0FFE0BB
:100B2000FFF1EEEEFFE0FBE0FFE1FAE1FFE0EAEECD
:100B3000FFE0EFEFFFFFF1EEE2FFE0FFE0EAF5FF9D
:100B4000E9EAF6130F01FE02020E3E0E0202FE005B
:100B5000F0F8FC049C9C9801403F20203F3C3F2043
:100B6000203F000F1F1F101F1F1F401028CEC17EE7
:100B700020702040C0800000000000000000000E37
:100B80006A59DBB9B9B9B247F9F1FAFCBC9E122235
:100B90003A0A0400000001061830F0787F2FCF10C9
:100BA0001108070000000000000000000000000322
:100BB0000404030030C0000000000000000000003A
:100BC0000000000000000C7080011EE0000000002A
:100BD0000000000000000000000000000F00000105
:100BE0000000001028CEC17E20702040C080000090
:100BF000000000000000000E6A59DBB9B9B9B24725
:100C0000F9F1FAFCBC9E12223A0A04000000010627
:100C10001830F0787F2FCF10110807000000000077
:100C200000000000000000030404030000000000B6
:100C300000000000000000000000000000000000B4
:100C400000008082C4241229E9465C600000000094
:100C500000000000C0A0D0B0D030F76A5CB379FECD
:100C60003E03000000000000000000000F12F8E941
:100C70005C5C4D20311EFF78000000000000000089
:100C80000000000000003CFE3F1F18F010F83E1F5F
:100C90002F9E600000000000000000000000000027
:100CA0000101030201000001010100000000000039
:100CB0000000000000000000C0E0F0787C78FC78C4
:100CC0007870F0E0C00000000000000000000000AC
:100CD0000000000000000000C0F0F8FCFE31151F0D
:100CE000003E11152615113E001F1531FEFCF8F0CF
:100CF000C0000000000000000000000000003FFFF6
:100D0000FF7F3F1C1060A040848282828440A060EC
:100D1000901C3F7FFFFF3F0000000000000000002C
:100D2000000000008098FF7C787A7CFDEBFAE5C03B
:100D3000C0C0E5FAEBFD7C7A787CFF98800000006B
:100D40000000000000000000000304040404070584
:100D50000404050503010101030505040405070456
:100D60000404040300000000000000000000000074
:100D7000000000000000C0E0F0787C78FC7878701B
:100D8000F0E0C000000000000000000000000000D3
:100D9000000000000000C0F0F8FCFE3195DF40BE0E
:100DA0009195A69591BE40DF9531FEFCF8F0C0000C
:100DB0000000000000000000000000003FFFFF7F77
:100DC0003F1C1067AF4E9E9696969E4EAF67901C46
:100DD0003F7FFFFF3F000000000000000000000018
:100DE00000008098FF7C787A7CFDEBFAE5C0C0C0FB
:100DF000E5FAEBFD7C7A787CFF988000000000002B
:100E000000000000000000030404040407050404BB
:100E10000505030101010305050404050704040495
:100E200004030000000000000000000000000000BB
:100E30000000E03C0780F01C000000800000000083
:100E40000000E030103360C007000000F00E010029
:100E5000000000000000071FFEEEC7E6C4ECFCFC2B
:100E6000FE3923261800000000000F071F0F073F60
:100E70001F0F0F081000000000000000000000001D
:100E800000000000004030180C06824130180800B5
:100E900000000080E0B01070E020901030F8FCFA04
:100EA00072322414080000004020180C06030100D0
:100EB00080631614F77E3E2F47279FDFDF38FE72D0
:100EC0002721130C000000000000000001010302B4
:100ED000070A081F1430231F17180700000000001E
:100EE000000000000000000000C020782E2264E412
:100EF000F8C0F8EC2253193B4E800000000C7751EB
:100F0000B3B9B9B8B2C5F8F9BFBF1F0E1E7FBF0E87
:100F1000C4380000000000000001070910120B0790
:100F200000000000010000000000000000000000C0
:100F300000000000780E00E03C070000788498D0A4
:100F4000E05A143A969AA69E2CC8B0F08B1008B0BE
:100F5000C0804063A76FFE0F050A0A0AC5FEFFCFD7
:100F600087030101000000030404040303020202DA
:100F70001B2F271717150800000000000000008035
:100F800040201018080000000000000000000000D1
:100F900000000000806026739010180CC2A2D0B030
:100FA000D030F060408000000000000000DDAAE3C7
:100FB00022BDF0F0EF12F8E95C5C4D20311EFF78A5
:100FC00000000000000001020203020101013CFEDA
:100FD0003F1F18F010F83E1F2F9E60000000000019
:100FE00000000000000000000101030201000001F8
:100FF000010100000000000010100010E8485B2014
:10100000000000000000000000001C0F0C000000A9
:1010100000000000000000000000182CE52C180063
:101020000000000000000000000000000F060000AB
:1010300000000000000000000000205B48E83000D5
:101040000000000000000000000000000000071C7D
:101050000C00000000000000000006090D0E10202A
:1010600040E0400000000000000000000000000020
:1010700000000000000000000000FFFFFFFFFFFF76
:10108000FFFFFFFFFFFFFFFFFFFFFFFFFFFFFFFF70
:10109000FFFFFFFFFFFFFFFFFFFFFFFFFFFFFFFF60
:1010A000FFFFFFFFFFFFFFFFFFFFFFFFFFFFFFFF50
:1010B000FFFF9B4100000000000000000000000056
:1010C00000008000000000000000881031E7FFFFF2
:1010D000FFFFFFFFFFFFFFFFFFFFFFFFFFFFFFFF20
:1010E000FFFFFFFFFFFFFFFFFFFFFFFFFFFFFFFF10
:1010F000FFFFFFFFFFFFFFFFFFFFFFFFFFFFFFFF00
:10110000FFFFFFFFFFFFFFFFFFFFFFFFFFFFFFFFEF
:10111000FFFFFFFFFFFFFFFFFFFFFFFFFFFFFFFFDF
:10112000FFFFFFFFFFFFFFFFFFFFFFFFFFFFFFFFCF
:10113000FFFFFFFFFFFFFFFFFFFFFFFFFFFFFFFFBF
:10114000FFFFFFFFFFFFFFFFFFFFFFFFFFFFFFFFAF
:10115000FFFFFFFCF8FEFFF6F0F8FCFEFCF8FEFCDB
:10116000F8FEF7F3F0E8E0E0C08000091E27E3F3A3
:10117000FFFFFFFFFFFFFFFFFFFFFFFFFFFFFFFF7F
:10118000FFFFFFFFFFFFFFFFFFFFFFFFFFFFFFFF6F
:10119000FFFFFFFFFFFFFFFFFFFFFFFFFFFFFFFF5F
:1011A000FFFFFFFFFFFFFFFFFFFFFFFFFFFFFFFF4F
:1011B000FFFFFFFFFFFFFFFFFFFFFFFFFFFFFFFF3F
:1011C000FFFFFFFFFFFFFFFFFFFFFFFFFFFFFFFF2F
:1011D000FFFFFFFFFFFFFFFFFFFFFFFFFFFFFFFF1F
:1011E000FFFFFFFFFFFFFFFFFFFFFFFFFFFFFFFF0F
:1011F000FFFFFFFFFFFFFFFFFFFFFFFFFFFFFFFFFF
:10120000FFFFFFFFFFFFFFFFFFFF7EBC78408081F5
:101210008387070F0F1F3F1F1F0F7F1F7F3FBF7F5A
:101220003F3F7F3F3F3F3F3F3F3F7FFFFFFF7F7F8E
:101230007FFF7F7FFFFFFFFFFFFFFFFFFFFFFFFF3E
:10124000FFFFFFFFFFFFFFFFFFFFFFFFFFFFFFFFAE
:10125000FFFFFFFFFFFFFF7FFFFFFFFFFFFFFFFF1E
:10126000FFFFFFFFFFFFFFFFFFFFFFFFFFFFFFFF8E
:10127000FFFFFFFFFFFFFFFFFFFFFFFFFFFFFFFF7E
:10128000FFFFFFFFFFFFFFFFFFFFFFFFFFFFFFFF6E
:10129000FFFFFFFFFFFFFFFFFFFFDF5F8F0F170F56
:1012A00003070B070301000100000000000001001C
:1012B000C0808080C0800000C0800080C001838327
:1012C00046468CC460606173628000103020220644
:1012D000060C0801022123434703050D0B070F07E6
:1012E0000B1B372F2F1F1F3F3F3F7F7F7F7F7F7F4E
:1012F0007F7F3726010103000001FFFFFFFFFFFF93
:10130000FFFFFFFFFFFFFFFFFFFFFFFFFFFFFFFFED
:10131000FFFFFFFFFFFFFFFFFFFFFFFFFFFFFFFFDD
:10132000FFFFFFFFFFFFFFFFFFFFFFFFFFFFFFFFCD
:10133000FFFFFFFFFFFFFFFFFFFFFFFFFFFEFFF8C5
:10134000FEF8FCFEFCF8FEFCF8FEF0F8FCFFFFFFE8
:10135000FFFFFFFFFFFFFFFFFFFFFFFFFFFFFFFF9D
:10136000FFFFFEEAD0E0E0C000000000061EBFFF65
:10137000FFFEFEFE30047CF8F8F0E0E0C0D0603202
:101380002266E4C0C0808000000000000000000071
:1013900000000000000000000000331101010341C3
:1013A0006123131303030B09191101018383010145
:1013B0004163231192920201010101A1E1F1FFFFBA
:1013C000FFFFFFFFFFFFFFFFFFFFFFFFFFFFFFFF2D
:1013D000FFFFFFFFFFFFFFFFFFFFFFFFFFFFFFFF1D
:1013E000FFFFFFFFFFFFFFFFFFFFFFFFFFFFFFFF0D
:1013F000FFFFFFFFFFFFFFFFFFFFFFFFFFFFFFFFFD
:10140000FFFFFFFFFFFFFBD8E4E0F0F8FCF9FFFF70
:10141000FFFFFFFFF8E6C48CFDFFFF7C70006060FB
:1014200060E4C5C4CCC0989080800000202060405B
:10143000800020C0800000000000FEFDFC3EDF9E1A
:10144000DEDEEEEFEEE6F68CBD7CFEFFFFFFFFFE7C
:10145000FEFEFFFFFFFFFF619C61FFFFFFFFFFFF3D
:10146000FFFFFFFFFFFFFFFFFFFFFFFFFFFFFFFF8C
:10147000FFFFFFFFFFFFFFFFFFFFFFFFFFFFFFFF7C
:10148000FFFFFFFFFFFFFFFFFFFFFFFFFFFFFFFF6C
:10149000FFFFFFFFFFFFFFFFFFFFFFFFFFFFFFFF5C
:1014A000FFFFFFFFFFFFFFFFFFFFFFFFFFFFFFFF4C
:1014B000FFFFFFFFFFFFFFFFFFFFF8FC3E80FEFC8A
:1014C000FCFCFFFFFFFFFFFFFFFFFFFFFE00FCF83C
:1014D000F0C000000F000070C080FFFFFFCFC0838E
:1014E0001D7DF1FE98961298DAE7FFFFFFFFFFFFE0
:1014F000FFFFFFFFFFFFFFFCC318DF3FFFFFFFFF02
:10150000FFFFFFFFFFFFFFFFFFFFFFFFFFFFFFFFEB
:10151000FFFFFFFFFFFFFFFFFFFFFFFFFFFFFFFFDB
:10152000FFFFFFFFFFFFFFFFFFFFFFFFFFFFFFFFCB
:10153000FFFFFFFFFFFFFFFFFFFFFFFFFFFFFFFFBB
:10154000FFFFFFFFFFFFFFFFFFFFFFFFFFFFFFFFAB
:10155000FFFFFFFFFFFFFFFFFFFFFFFF00FFFFFF9A
:10156000FFFFFFFFFFFFFFFFFFFFFFFF03F8FFFF8E
:10157000FFFF9F8000101030E1C33F1F7F0FE38CFF
:1015800062606090FC7CE3370F37078FFFFFFF7FBF
:101590007FFFFFFFFFFFFFFFFFFEFDF0876F6F9FE5
:1015A000FFFFFFFFFFFFFFFFFFFFFFFFFFFFFFFF4B
:1015B000FFFFFFFFFFFFFFFFFFFFFFFFFFFFFFFF3B
:1015C000FFFFFFFFFFFFFFFFFFFFFFFFFFFFFFFF2B
:1015D000FFFFFFFFFFFFFFFFFFFFFFFFFFFFFFFF1B
:1015E000FFFFFFFFFFFFFFFFFFFFFFFFFFFFFFFF0B
:1015F000FFFFFFFFFFFFFFFFFFFFFFFF00FFFFFFFA
:10160000FFFFFFFFFFFFFFFFFFFFFFFF00F9F8F8FD
:10161000FCFEFFFFFFFFF6E0C187000000010001B4
:1016200001010505060200000482C3C1E0F0F0F8E4
:10163000F8FEFEFDFDF3E7CFDFDFDFDFDFBF7FFF7B
:10164000FFFFFFFFFFFF7F7F7F7F7F7FFFFFFFFFAA
:10165000FFFFFFFFFFFF7F7F7F7F7F7F7F7F7F7F9A
:101660007FFFFF7F7F7F7F7F7F7FFFFF7F7F7F7F8A
:10167000FFFFFFFF7F7F7FFFFFFFFFFFFFFF7F7FFA
:101680007F7F7F7FFFFFFF7FFFFF7F7F7F7F7FFF6A
:10169000FFFF7F7F7F7FFF7F7F7F1FC0FE7F3F3FFA
:1016A0007F7FFFFFFFFFFFFFFFFFFFFF00FFFFFF49
:1016B000FFFFFFFFFFFFFFFFFFFFF8FCF0E0FCFC78
:1016C000FCFFFDFBFAF8FCFEFFFFFFFFFFFFFFFF43
:1016D000FFFFFFFFFFFFFFFFFFFFE7C74F87908E72
:1016E000CCEDFDFCFEFEFEFEFFC6E2F2FAFEF2E0ED
:1016F000E1C5FDFCFEFEFEFFFFFFF9D88880C0C0FB
:101700008080C0828686D4909000B0A0A0C0C0E443
:10171000E4C4C48C8C88C0C080800000880810900D
:10172000108084C4C0C4848080802090901468801D
:1017300088880800000080008000C080008080D081
:10174000FCFCFFFFFFFFDFE7E3E3E307E0FFFFFF52
:10175000FFFFFFFFFFFFFFFFFFFFFFFFFFFFFFFF99
:10176000FFFFFFFFFFFFFFFFFFFFFFFFFFFFFFFF89
:10177000FFFFFFFFFFFFFFFFFFFFFFFF807FFFFF78
:10178000FFFFFFFFFFFFFFFFFFFFFFFFFFFFFFFF69
:10179000FFFFFFFFFFFFFFFFFFFFFFFFFFFFFFFF59
:1017A000FFFFFFFFFFFFFFFFFF807FFFFFFFFFFF48
:1017B000FFFFFFFFFFFFFFFFFFFFFFFEFEFEFF3FFC
:1017C00080FFFFFFFFFFFFFFFFFFFFFEFEFEFFFFAB
:1017D000FFFFFFFEFEFFFFFFFEFFFFFF807FFFFF1B
:1017E000FFFFFFFFFFFFFFFFFFFF01FCFFFFFFFF0A
:1017F000FFFFFFFF7F7F7F7F7FFFFFFFFFFFFFFF79
:10180000FFFFFFFFFFFFFFFFFFFFFFFFFFFFFFFFE8
:10181000FFFFFFFFFFFFFFFFFFFFFFFFFFE0CF8F97
:101820008F9FFFFFFFFFFFFFFFFFFFFFFFFFFFFF98
:10183000FFFFFFFFFFFFFFFFFFFFFFFFFFFFFFFFB8
:10184000FFFFFFFFFFFFFFFFFFFFF0E7C7C7CFFF6F
:10185000FFFFFFFFFFFFFFFFFFFFFFFFFFFFFFF0A7
:10186000E7C7C7CFFFFFFFFFFFFFFFFFFFFFFFFF40
:10187000FFFFFFFFFFFFFFFFFFFFFFFFFFE0CF8F37
:101880008F9FFFFFFFFFFFFFFFFFF0E7C7C7CFFFFF
:10189000FF7F3713010100000000FFFFFFFFFFFF84
:1018A000FFFFFFFFFFFFFFFFFFFFFFFFFFFFFFFF48
:1018B000FFFFFFFFFFFFFFFFFFFFFFFFFFFFFFFF38
:1018C000FFFFFFFFFFFFFFFFFFFFFFFFFFFFFFFF28
:1018D000FFFFFFFFFFFFFFFFFFFFFFFFFFFFFFFF18
:1018E000FFFFFFFFFFFFFFFFFFFFFFFFFFFFFFFF08
:1018F000FFFFFFFFFFFFFFFFFFFFFFFFFFFFFFFFF8
:10190000FFFFFFFFFFFFFFFFFFFFFFFFFFFFFFFFE7
:10191000FFFFFFFFFFFFFFFFFFFFFFFFFFFFFFFFD7
:10192000FFFFFFFFFFFFFFFFFFFFFFFFFFFFFF7B4B
:101930001C0C0E02000000000000FF7FFFFF7FFF75
:10194000FF7FFFFFFFFFFFFFFFFFFFFFFFFFFFFF27
:10195000FFFFFFFFFFFFFFFFFFFFFFFFFFFFFFFF97
:10196000FFFFFFFFFFFFFFFFFFFFFFFFFFFFFFFF87
:10197000FFFFFFFFFFFFFFFFFFFFFFFFFFFFFFFF77
:10198000FFFFFFFFFFFFFFFFFFFFFFFFFFFFFFFF67
:10199000FFFFFFFFFFFFFFFFFFFFFFFFFFFFFFFF57
:1019A000FFFFFFFFFFFFFFFFFFFFFFFFFFFFFFFF47
:1019B000FFFFFFFFFFFFFFFFFFFFFFFFFFFFFFFF37
:1019C000FFFFFFFFFFFFFFFFFFFFFFFFFFFFFFFC2A
:1019D000CEE27010000000000000000001000003D3
:1019E00000000301496D3FFF7F3FFFFFFFFFFFFF47
:1019F000FFFFFFFFFF7F7F7F7FFF7F7F7F7FFFFFF7
:101A0000FF7F7F7FFFFFFFFFFFFFFFFFFFFFFFFF66
:101A1000FFFFFFFFFFFFFFFFFFFFFFFFFF7F7F7F56
:101A20007FFF7F7F7FFFFFFFFFFF7F7F7F7F7F7FC6
:101A3000FFFFFFFF7F7F7F7FFFFF7F7F7F7F7F7FB6
:101A40007FFFFF7F7F7FFFFFFFFFFFFFFF7F7F7F26
:101A50007FFF7F7F7FFF7F7F7FFFFFFFFF7F7F7F96
:101A60007F7F7FFFFFFFFF7F7FFFFFFFFF7F7F7F86
:101A70007FFF7E5B490000000000000000000000C6
:101A800000000000000000000000000000103031E5
:101A900021210808080C0C1C18180C0C1810000048
:101AA00008181000080819393810100020203019C3
:101AB000191101010101111018080808080C0C1C6B
:101AC00018181018080800000000000000000008A6
:101AD000080C0C0C040400101018183830301010CA
:101AE000000000000818180808010808080C0C1C61
:101AF000181808080000000004040070400E1818B0
:101B0000190E40300000000008080808080C0C1CE2
:101B100018180000000000000000080B000202027C
:101B20000000090400000102020000052400100169
:101B3000052401010104240206052406000107050D
:101B4000810310004009040100020A00000007059B
:101B5000020240000007058302400000040309045C
:101B600012010002EF020140412336800001010210
:101B7000030141726475696E6F204C4C43004172E1
:101B80006475696E6F204C656F6E6172646F0000E2
:101B9000611F11241FBECFEFDAE0DEBFCDBF11E021
:101BA000A0E0B1E0EAE3FCE602C005900D92AE379A
:101BB000B107D9F727E0AEE7B1E001C01D92A23628
:101BC000B207E1F71DE0C9ECDDE004C02197FE019A
:101BD0000E942334C83CD107C9F70E94981F0C9477
:101BE0001B360C940000809197010895CF92DF92EC
:101BF000EF92FF92CF93DF93EC016A017B01E091BA
:101C00004C07F0914D0709958823F1F18091FB066F
:101C10008230D0F181E08093FA068091F9068093BA
:101C2000F80680918100887F816080938100DE01C9
:101C3000AA0FBB1FA70196010E94C33228EE33E012
:101C400040E050E00E940D3369017A019E0150E0AE
:101C500040E060E072E18AE790E00E94A432215007
:101C60003109410951093093890020938800C092BD
:101C7000F406D092F506E092F606F092F70680910F
:101C80006F00826080936F00DF91CF91FF90EF90A3
:101C9000DF90CF9008956F927F928F929F92AF9234
:101CA000BF92CF92DF92EF92FF920F931F93CF9349
:101CB000DF93DC01FA011491319654913196C12FD2
:101CC000D0E0222309F1CC24C394D12C852F877036
:101CD00011F4D12CC12CE52EE694E694E694EC0C9C
:101CE000FD2CF11CEC9EC001ED9E900DFC9E900D14
:101CF0001124033011F4880F991F289F7001299F28
:101D0000F00C1124EE0DFF1D7D01EC0EFD1E1E14C6
:101D10001F040CF06BC0A038B1050CF067C0CB01FC
:101D2000850F911D181619060CF060C060347105FE
:101D30000CF05CC0309709F459C0362F3770CB01D6
:101D400077FD079623E0959587952A95E1F7282F4B
:101D500077FF04C0332311F02FEF280F6627772772
:101D60006A1B7B0BB7FD02C070E060E090E89A1B35
:101D700040E8E416F1040CF4912F961BE22E022E9B
:101D8000000CFF08DE2CD0942F3F0CF0D12C41E04A
:101D9000852F877009F440E0B52EB694B694B694BA
:101DA0004B0DE40EF11C89E0E816F10414F048E054
:101DB000421BB42EBD182D0D40E8240370011124E0
:101DC000AE0DBF1DA60FB71F1D9D600D711D112407
:101DD000AF01460F571FC32E032E000CDD08033042
:101DE00009F4C7C090F4023009F474C0DF91CF91B8
:101DF0001F910F91FF90EF90DF90CF90BF90AF9029
:101E00009F908F907F906F9008950A3FA1F1B20E3E
:101E10000B3F61F72B1551F3BD016C507D4F10E066
:101E200000E0091708F09FC0FA01E00FF11FE491EC
:101E3000F0E04F010C2C02C0880C991C0A94E2F7C8
:101E400027FD06C0FB018081F82CF0948F21808350
:101E5000332361F0273054F47B01F0E8EF0EF11CDE
:101E6000A92CA094F70180818A2180830F5F1F4FE6
:101E70006F5F7F4FD6CFB20E2B1509F4B7CFBD01E0
:101E80006C507D4F10E000E0091708F066C0FA01C1
:101E9000E00FF11FE491F0E04F010C2C02C0880C20
:101EA000991C0A94E2F727FD04C0FB018081882970
:101EB0008083332351F0273044F47B01F0E8EF0EA8
:101EC000F11CF7018081892980830F5F1F4F6F5FAD
:101ED0007F4FDACF6FEF70E0032E02C0660F771FDF
:101EE0000A94E2F760957095972E8B2C820E281538
:101EF00009F47CCF8D010C501D4FF12CE12CE9161B
:101F000030F5FA01EE0DFF1DE491F0E03F010C2CDD
:101F100002C0660C771C0A94E2F727FD05C0F801A1
:101F20008081862386298083332359F027304CF41F
:101F30005801F0E8AF0EB11CF50180818921872995
:101F40008083FFEFEF1AFF0A0F5F1F4FD8CF2F5F7D
:101F50004C0F5D1FA058BF4FCACF2F5F4C0F5D1FA6
:101F6000A058BF4F89CF2F5F4C0F5D1FA058BF4FA8
:101F700051CFE92EF12CFA01E60FF71FAC50BD4FFF
:101F800060E870E06E197F09CE19DF098E01000F3D
:101F9000111F41E050E07A01032E01C0EE0C0A94BB
:101FA000EAF7592F4B2D892E932ECF93DF93ED0116
:101FB000EF96EF962296A590C590992059F0AE9C89
:101FC0005001CE9C600127302CF4F880D094FD2085
:101FD000FB28F99222233AF0FC90C094FC20FA28C6
:101FE000FD920C94F40F11965A9529F74A9551F0E9
:101FF000582D23951124E00FF11DA60FB11DC60F1A
:10200000D11DD9CFDF91CF911124F0CEE4EFF2E0D2
:1020100080E0A0E0B8E000800EBC8111012C119797
:10202000A0FDFDCF0192B9F70DB40895E4EFF2E001
:1020300081118FEF00248193819381938193039485
:10204000D1F70895FC013D96019620E032913111BF
:102050002F5FE817F907D1F7222341F044E150E060
:1020600060E070E080E296E00C94F60D0895FC01CB
:102070008091F302882311F13FB7F89482E08093B6
:10208000E9002091F200822F90E01816190614F44E
:1020900081E090E0882339F0289844E64093F202EA
:1020A0004091F1004083222339F02091F200211168
:1020B00003C02BE62093E8003FBF08958FEF9FEF0A
:1020C00008952FB7F89483E08093E9009091E80099
:1020D000892F807295FF04C09091F20080E4891BE3
:1020E0002FBF08958091EA0281110DC082E0809394
:1020F000E60284E08093E7021092E9021092E8027F
:1021000081E08093EA0286EE92E00895CF93DF9318
:102110001F92CDB7DEB76983DC01ED91FC9102809F
:10212000F381E02D41E050E0BE016F5F7F4F0995E4
:102130000F90DF91CF91089583E08093E900809123
:10214000F200882319F08AE38093E80008950E9442
:10215000611090E00895CF93DF931F92CDB7DEB763
:10216000FC018485958597FD08C02FEF3FEF3587EB
:1021700024870F90DF91CF910895CE0101960E94A0
:102180003710019719F4898190E0F3CF8FEF9FEF1B
:10219000F0CF0F931F93CF93DF931F92CDB7DEB78E
:1021A0008C01FC018485958597FF0BC0CE010196BB
:1021B0000E943710019771F4898190E0F8019587AA
:1021C0008487F801848595850F90DF91CF911F91C9
:1021D0000F9108958FEF9FEFF1CFFC0184859585D6
:1021E00097FD0BC09FB7F89482E08093E90080913F
:1021F000F2009FBF90E0019608959FB7F89482E0A7
:102200008093E9008091F2009FBF90E00895409193
:10221000E0025091E1022091DE023091DF0242178C
:102220005307B4F49091E8009570E1F39091E800C1
:1022300092FD19C08093F1008091E0029091E1023B
:1022400001968F739927892B19F48EEF8093E800FC
:102250008091E0029091E10201969093E1028093D7
:10226000E00281E0089580E00895EF92FF920F93DD
:102270001F93CF93DF93F82E192FE62E042F81E0C2
:10228000860F880F0E94071183E00E940711CF2D4F
:10229000D12FEC0EFD2EF11CCE15DF05B9F007FF96
:1022A00013C0FE0184910E940711182F80E00E9444
:1022B0000711812321968111EFCFDF91CF911F91DB
:1022C0000F91FF90EF9008958881EDCF81E0F5CFD9
:1022D000DF92EF92FF920F931F93CF93DF93D82E4D
:1022E0008A01EB017B01E40EF51ECE15DF0559F0E6
:1022F000D7FE12C0FE0184910E9407112196811120
:10230000F4CF0FEF1FEFC801DF91CF911F910F9115
:10231000FF90EF90DF9008958881EECF0F931F9389
:10232000CF93DF931F92CDB7DEB782E0898342E47B
:1023300050E06AE17BE180E80E9468110E9472101F
:10234000DC0112960D911C910115110589F0D8013F
:10235000ED91FC910280F381E02DBE016F5F7F4F14
:10236000C801099597FD04C0F80100851185ECCFDF
:1023700089810F90DF91CF911F910F910895615046
:1023800030F02091F100FC0120830196F8CF2898CD
:1023900084E68093F202089508953FB7F8948091FF
:1023A000930190919401A0919501B091960126B569
:1023B000A89B05C02F3F19F00196A11DB11D3FBF7D
:1023C000BA2FA92F982F8827BC01CD01620F711D4C
:1023D000811D911D42E0660F771F881F991F4A9546
:1023E000D1F708958F929F92AF92BF92CF92DF92D2
:1023F000EF92FF926B017C010E94CD114B015C01B9
:10240000C114D104E104F104B9F00E94CD1168199E
:1024100079098A099B09683E73408105910580F31B
:1024200021E0C21AD108E108F10888EE880E83E0A5
:10243000981EA11CB11CE4CFFF90EF90DF90CF90CD
:10244000BF90AF909F908F9008958F929F92AF9280
:10245000BF92CF92DF92EF92FF920F931F93CF9391
:10246000DF936C017B018A0180910E01882309F4BE
:102470005CC08091F302882309F457C08091E50283
:1024800080FF05C08091E00082608093E000E80159
:10249000B12C8AEFA82E93E0892E2AE3922E209762
:1024A00011F4BB20D9F10E94611081110AC0AA94D5
:1024B000AA20D9F161E070E080E090E00E94F21182
:1024C000EECF8C171D0611F00CF08C2F9FB7F894EF
:1024D0008092E9002091E80025FD02C09FBFDFCF78
:1024E000282F30E0C21BD30BF701815020F041911F
:1024F0004093F100FACFE20EF31EBB2021F0909240
:10250000E800B12CEBCF8091E80085FDE7CF9092F9
:10251000E800BB24B394209709F3F3CF5D9884E6D9
:102520008093E402101611063CF081E090E0F60181
:102530009383828310E000E0C801DF91CF911F9167
:102540000F91FF90EF90DF90CF90BF90AF909F9052
:102550008F900895CF92DF92EF92FF921F93CF93C7
:10256000DF93E82FF0E0E35EFE4F1081E62FF0E00E
:10257000603398F5E452F54FE491CE2FD0E0F12C82
:10258000E12C60E074E284EF90E0A7019E010E94DC
:10259000A432215031094109510991E02115310539
:1025A00081E0480751056CF060E970ED83E090E050
:1025B000A7019E010E94A43221503109410951090D
:1025C00093E0113089F0133039F1DF91CF911F91F1
:1025D000FF90EF90DF90CF900895EE0FFF1FE45231
:1025E000F64FC591D491CBCF8091FA068111EDCFF2
:1025F00080918100887F892B8093810030938900AE
:1026000020938800109285001092840080916F00C2
:10261000826080936F00D9CF80919100887F892B51
:102620008093910030939900209398001092950028
:1026300010929400D0939101C093900181E0809317
:102640008F0180917100826080937100BECFE82F6E
:10265000F0E0E35EFE4F8081813019F08330A9F015
:1026600008958091FA0681110FC080916F008D7FCF
:1026700080936F0080918201E0918001F09181014F
:102680009081809589238083089510928F01809195
:10269000F8068111F9CF80918D01E0918B01F091C5
:1026A0008C01EECF9091FB06923009F471C0292F76
:1026B00030E0F901E35EFE4F408122583E4FF901C0
:1026C0008083913031F420917E01281302C09093D1
:1026D00083019F5F9093FB0690E0FC01E35EF54F62
:1026E00024918250964FFC01849130E0220F331FD9
:1026F000F901E051F64F65917491F901EE51F64FF1
:10270000A591B4919C91982B9C93413019F0433042
:10271000D9F0089590916400977F9093640010928F
:1027200080001092810090918100986090938100C8
:1027300090918100916090938100709381016093EA
:10274000800180938201089590916500977F909316
:102750006500109290001092910090919100986005
:10276000909391009091910091609093910070935B
:102770008C0160938B0180938D018091FB068823EF
:1027800021F06CE380E00E94AA1280E00C942713F1
:1027900008950F930BEF0E944B0E0F910895BC010B
:1027A00090E080E00C94F2118FB18095807F669B61
:1027B00088601C9B846008953F924F925F926F9255
:1027C0007F928F929F92AF92BF92CF92DF92EF92C1
:1027D000FF920F931F93CF93DF9330E0F901E80F3F
:1027E000F91FF7FDBFC0803891050CF0BBC0FB019D
:1027F000E00FF11DF7FDB6C0603471050CF0B2C0FA
:10280000DB0177FF04C0AA27BB27A61BB70BA77065
:10281000BB27FB0177FD3796C3E0F595E795CA9591
:10282000E1F777FF07C0319768E070E0EB01CA1B62
:10283000DB0BDE01402E469446944694512C0770E3
:1028400019F0DFEF4D1A5D0ABF01EF01D695DC2FBD
:10285000CC27D795C795C80FD91FCC50DD4F8A011B
:10286000460E571E48E050E04A018A1A9B0A461657
:10287000570609F477C06830710509F473C06F3FDB
:10288000EFEF7E070CF44BC06C0150E040E03E01DE
:10289000E0E86E0E711CD7FC35C06F3F760709F477
:1028A0005DC05E01A40EB51EF501F080F801E40FD5
:1028B000F51F33243394E31039C0E4910A2E01C08C
:1028C000EE0F0A94EAF7FE2AF501F0821097D1F094
:1028D00067307105B9F05301A40EB51EF501F08003
:1028E000F801E40FF51F33243394E3102BC0E49177
:1028F000F0E0082C02C0F595E7950A94E2F7FE2A6D
:10290000F501F0824F5F5F4FFFEFCF1ADF0A4217EA
:1029100053072CF4F0E8CF16D10409F0BCCF6F5F59
:102920007F4FC058DF4F020F131FA1CFE491F0E09B
:102930000A2E02C0EE0FFF1F0A94E2F7E095F09511
:10294000FE22C2CFE491F0E0082C02C0F595E79595
:102950000A94E2F7E095F095FE22D2CF109709F0A5
:10296000BACFD0CFDF91CF911F910F91FF90EF9011
:10297000DF90CF90BF90AF909F908F907F906F909F
:102980005F904F903F9008950895CF93DF93C0914B
:10299000D602D091D702219644E150E060E070E089
:1029A00080EE96E00E94F60DCE01DF91CF91089562
:1029B000EF92FF920F931F93CF93DF9323EBE22EBF
:1029C00022E0F22EC8E0D2E08E01F70181917F0172
:1029D0008823B9F0F801618180915D07082E000C11
:1029E000990B680F792F711D30818091DA02082EC2
:1029F000000C990B22814EE558E0830F911D0E9437
:102A0000C913095F1F4FF0ECEF16F2E0FF06E9F67D
:102A100005EA12E0F80181918F018823B1F0698104
:102A200080915D07082E000C990B680F792F711D9E
:102A300038818091DA02082E000C990B2A814EE52C
:102A400058E0830F911D0E94C9132796F2E0023BC4
:102A50001F0701F79CE9E92E92E0F92EC0EDD1E0C5
:102A60008E01F70181917F018823B9F0F80161811E
:102A700080915D07082E000C990B680F792F711D4E
:102A800030818091DA02082E000C990B228140E4FB
:102A900059E0830F911D0E94C913095F1F4FF4EA8B
:102AA000EF16F2E0FF06E9F603E912E08BE9E82E03
:102AB00082E0F82EF80181918F018823B1F06981BD
:102AC00080915D07082E000C990B680F792F711DFE
:102AD00038818091DA02082E000C990B2A8140E49B
:102AE00059E0830F911D0E94C9132796E016F10645
:102AF00009F7DF91CF911F910F91FF90EF9008950B
:102B00002091DC023091DD02C90160E370E00E9497
:102B10000334892B29F48091D1028F5F8093D102F5
:102B2000C9016CE070E00E940334892B09F055C0A4
:102B300080918702811119C0E0ECF2E0DF018E91F3
:102B40009081FD01908381831092C002A35BB2400B
:102B5000A9F783EB92E00E942210809187028F5F99
:102B60008430C8F5809387020895813081F4E2EBC8
:102B7000F2E0DF018E919081FD01908381831092BC
:102B8000B202A55AB240A9F785EA92E0E4CF8230BA
:102B900081F4E4EAF2E0DF018E919081FD019083FF
:102BA00081831092A402AC59B240A9F78CE992E05B
:102BB000D2CF833091F6EBE9F2E0DF018E91908184
:102BC000FD019083818310929B02A359B240A9F723
:102BD00083E992E0C0CF109287020895CF92DF92EE
:102BE000EF920F931F93CF93DF9313E08091C8026E
:102BF000813099F560915D07C62E660FDD08C091A2
:102C0000DA020C2E000CDD0BB601675E7F4FE12C63
:102C100005E02EE040E558E0CE018B599F4F0E9421
:102C2000DC13609199016C0D7D2D711D675F7F4FE5
:102C3000809198010CE02CE048E358E08C0F9D2F28
:102C4000911D0E94DC13115089F6DF91CF911F91E5
:102C50000F91EF90DF90CF900895823099F56091B9
:102C60005D07C62E660FDD08C091DA020C2E000C3F
:102C7000DD0BB601675E7F4FE12C05E02EE040E5FD
:102C800058E0CE018B599F4F0E94DC13609199014F
:102C90006C0D7D2D711D675F7F4F809198010CE059
:102CA0002CE048E358E08C0F9D2F911D0E94DC130F
:102CB0006091A0016C0D7D2D711D675F7F4F80912C
:102CC0009F01B9CF833009F0BECFC0905D070C2CB7
:102CD000000CDD08C091DA020C2E000CDD0BB601F1
:102CE000675E7F4FE12C05E02EE040E558E0CE0125
:102CF0008B599F4F0E94DC13609199016C0D7D2DC3
:102D0000711D675F7F4F809198010CE02CE048E3D4
:102D100058E08C0F9D2F911D0E94DC136091A00143
:102D20006C0D7D2D711D675F7F4F80919F012CE0A1
:102D300048E358E08C0F9D2F911D0E94DC13609199
:102D4000A7016C0D7D2D711D675F7F4F8091A601DE
:102D500072CFEF920F938091D802811117C06091CA
:102D60005D07062E000C770B645F7F4F8091DA02BF
:102D7000082E000C990BE12C05E226E24AE757E009
:102D800001960E94DC130F91EF9008958130D9F7DE
:102D90008091C102882319F3813091F460915D071D
:102DA000062E000C770B645F7F4F8091DA02082EAD
:102DB000000C990BE12C05E226E24CEB56E0E0CF4B
:102DC000823091F460915D07062E000C770B645FF2
:102DD0007F4F8091DA02082E000C990BE12C05E25E
:102DE00026E24EEF55E0CCCF833069F660915D0767
:102DF000062E000C770B645F7F4F8091DA02082E5D
:102E0000000C990BE12C05E226E240E455E0B8CF36
:102E10008091DC029091DD0260E370E00E94033457
:102E2000892B31F49091D80281E0891B8093D802DC
:102E300008958091DC029091DD0268E170E00E94CB
:102E40000334892B51F4809185028F5F87301CF405
:102E50008093850208951092850208955F926F9283
:102E60007F928F929F92AF92BF92CF92DF92EF921A
:102E7000FF920F931F93CF93DF930E94D413682E7A
:102E80000E94D413582E0E94D413782E0E94D4137B
:102E9000882E0E94D413982E0E94D41354FA5524DD
:102EA00050F8C52D90E0D92FCC0FDD1F262D660CD4
:102EB000330B2227330F221F3327C20FD31F75FA7C
:102EC000AA24A0F8B12CAA0CBB1CAA0CBB1CCA0DCE
:102ED000DB1D86FACC24C0F8D12C63E0CC0CDD1CC1
:102EE0006A95E1F7CC0DDD1D93FAEE24E0F8F12CA4
:102EF00074E0EE0CFF1C7A95E1F7CE0DDF1D82FB2E
:102F0000002700F910E0C801E5E0880F991FEA9555
:102F1000E1F78C0F9D1FDF91CF911F910F91FF90D3
:102F2000EF90DF90CF90BF90AF909F908F907F9069
:102F30006F905F900895EF920F938091000183301E
:102F400009F09BC08091D30281111AC060915D0786
:102F5000062E000C770B6B587F4F8091DA02082EFB
:102F6000000C990BE12C04E123E147E055E0459684
:102F70000E94DC131092DB0280EB80935C075DC043
:102F8000813099F460915D07062E000C770B6B5829
:102F90007F4F8091DA02082E000C990BE12C04E19E
:102FA00026E145EC54E08A96E3CF8230A1F46091AB
:102FB0005D07062E000C770B6B587F4F8091DA026D
:102FC000082E000C990BE12C04E124E149E854E0BF
:102FD0008E5B9F4FCDCF8330C9F460915D07062E85
:102FE000000C770B6B587F4F8091DA02082E000C93
:102FF000990BE12C04E125E14AE454E0865A9F4F05
:103000000E94DC138EED8093DB0217C08430F9F44C
:1030100060915D07062E000C770B6B587F4F8091F7
:10302000DA02082E000C990BE12C04E124E149E8B6
:1030300054E081599F4F0E94DC138091D202853069
:1030400019F48AE0809301010F91EF900895853083
:10305000A1F760915D07062E000C770B6B587F4F30
:103060008091DA02082E000C990BE12C04E126E194
:1030700048E054E08E579F4FDECF823009F08AC07F
:103080008091D302811117C060915D07062E000C5C
:10309000770B6F597F4F8091DA02082E000C990B45
:1030A000E12C02E120E148ED53E045960E94DC135B
:1030B0001092DB02C2CF813099F460915D07062E39
:1030C000000C770B6F597F4F8091DA02082E000CAD
:1030D000990BE12C03E126E146E953E08996E6CF1E
:1030E0008230A1F460915D07062E000C770B6F59BA
:1030F0007F4F8091DA02082E000C990BE12C02E13F
:103100002FE049E653E08E5B9F4FD0CF833091F4A0
:1031100060915D07062E000C770B6E597F4F8091F2
:10312000DA02082E000C990BE12C01E120E149E3C1
:1031300053E064CF8430A1F460915D07062E000C4B
:10314000770B6C597F4F8091DA02082E000C990B97
:10315000E12C02E125E14AEF52E084599F4F6BCF09
:10316000853009F06ACF60915D07062E000C770B61
:10317000635A7F4F8091DA02082E000C990BE12CE4
:1031800004E124E14EEB52E081589F4F0E94DC1392
:103190008EEAF3CE813009F092C08091D302823062
:1031A000C9F460915D07062E000C770B6C5B7F4FB6
:1031B0008091DA02082E000C990BE12C04E121E148
:1031C0004BE852E08C5B9F4F0E94DC131092DB02B5
:1031D00087EED3CE8330C9F460915D07062E000CD4
:1031E000770B6B5B7F4F8091DA02082E000C990BF6
:1031F000E12C03E123E142E552E0885A9F4F0E940F
:10320000DC138EED8093DB02E3CF843091F4609188
:103210005D07062E000C770B6C5B7F4F8091DA0206
:10322000082E000C990BE12C03E124E146E152E069
:1032300094CF853009F001CF60915D07062E000C18
:10324000770B6B5B7F4F8091DA02082E000C990B95
:10325000E12C03E124E14AED51E08F579F4F0E949A
:10326000DC13B6CF8330A1F460915D07062E000C0D
:10327000770B645D7F4F8091DA02082E000C990B6A
:10328000E12C07E126E149E551E0895A9F4FB8CE8C
:10329000843009F0D2CE60915D07062E000C770BCA
:1032A000605D7F4F8091DA02082E000C990BE12CB3
:1032B00004E12FE04CE251E080599F4FD0CF8111C3
:1032C000BCCE8091D302823069F660915D07062EF4
:1032D000000C770B605D7F4F8091DA02082E000CA6
:1032E000990BE12C02E125E14BE951E00CCF40E5DF
:1032F00050E060E070E08CE69CE00E94F60D64E631
:1033000070E080E090E00E94F21140E550E060E063
:1033100070E08DE49AE00E94F60D64E670E080E0D3
:1033200090E00C94F2110F931F93CF93DF930AEC6C
:1033300012E0CDEAD1E0F80181918F018823B1F04C
:10334000698180915D07082E000C990B680F792F19
:10335000711D38818091DA02082E000C990B2A81A8
:103360004AEE50E0830F911D0E94C9132796F2E0A8
:103370000E3C1F0701F7DF91CF911F910F91089528
:10338000FC0180819181009711F00C94C53408955F
:10339000EF92FF920F931F93CF93DF93EC017B018A
:1033A0008A0188819981009729F02A813B8124171D
:1033B000350788F4B8016F5F7F4F0E944E35009744
:1033C00091F0998388831B830A832C813D81232B71
:1033D00011F4FC0110821D830C83B701888199814F
:1033E0000E9414360CC088819981009711F00E94C8
:1033F000C534198218821D821C821B821A82CE015A
:10340000DF91CF911F910F91FF90EF9008955F9200
:103410006F927F928F929F92AF92BF92CF92DF92E4
:10342000EF92FF920F931F93CF93DF93CDB7DEB749
:103430006D970FB6F894DEBF0FBECDBF8091D60258
:103440009091D7021B8A1A8A1D8A1C8A1F8A1E8A9B
:103450004AE09E012F5F3F4F6901B9010E94693127
:10346000F60101900020E9F73197AF014C195D0991
:10347000B601CE0142960E94C819AE88BF88198E47
:10348000188E1B8E1A8E1D8E1C8E50E040E06CE74D
:1034900071E0CE0148960E94C819BB248FEF9FE1CE
:1034A000A89E3001A99E700CB89E700C1124F12CBE
:1034B000E12CEA14FB040CF0A1C03FEFE31AF30A7D
:1034C000470181E0881A91081A8219821C821B82A6
:1034D0001E821D8250E040E06CE771E0C6010E9450
:1034E000C8198E899F898816990620F587018E153F
:1034F0009F0508F48C01EA89FB89E00FF11F5080D9
:1035000010826A897B89680D791D6115710509F43E
:1035100055C0FB0101900020E9F73197AF01461B30
:10352000570BC6010E94C8198A899B89080F191F69
:10353000F8015082888D998D009709F44EC06981F9
:103540007A816115710509F446C04A8D5B8D2D8124
:103550003E814217530708F43EC00E9414368D8105
:103560009E819D8F8C8F1E821D82C6010E94C01974
:10357000888D998D20E0009719F00E942D31262F1B
:1035800080915D07082E000C990BBC01665F7F4F90
:10359000C701860D971D33E0880F991F3A95E1F713
:1035A00089569F4F3091DA0202E04CEA50E0830FD7
:1035B000911D37FD9A950E944B0E7BCF89819A8190
:1035C000009711F00E94C5341A8219821E821D8252
:1035D0001C821B82A9CF0E94C53489819A81998F50
:1035E000888F8B819C819B8F8A8F8D819E819D8FFF
:1035F0008C8F1A8219821C821B82B5CFCE0148960D
:103600000E94C019CE0142960E94C0196D960FB655
:10361000F894DEBF0FBECDBFDF91CF911F910F9108
:10362000FF90EF90DF90CF90BF90AF909F908F90E2
:103630007F906F905F9008951F920F920FB60F9238
:1036400011248F939F938091E1009091E100937FEB
:103650009093E10083FF0FC01092E90091E09093F6
:10366000EB001092EC0092E39093ED001092F302C5
:1036700098E09093F00082FF22C093E09093E900DD
:103680009091F200992319F09AE39093E8009091B9
:10369000E402992341F09091E40291509093E40266
:1036A000911101C05D9A9091F202992341F090919D
:1036B000F20291509093F202911101C0289A84FF76
:1036C00018C08091E2008E7E81608093E20080913C
:1036D000E1008F7E8093E1008091E5028E7E806123
:1036E0008093E5029F918F910F900FBE0F901F90D6
:1036F000189580FFF7CF8091E2008E7E80618093E5
:10370000E2008091E1008E7E8093E1008091E502ED
:103710008E7E8160E5CF1F920F920FB60F9211241B
:10372000CF92DF92EF92FF920F931F932F933F93CD
:103730004F935F936F937F938F939F93AF93BF93B9
:10374000EF93FF93CF93DF93CDB7DEB76C97DEBFD8
:10375000CDBF1092E9008091E80083FF25C068E0AA
:10376000CE0145960E94BF1182EF8093E8008D89BB
:1037700087FF39C09091E80090FFFCCF982F90769A
:1037800009F034C19E894F89588D2F89F88C911189
:1037900031C0803861F58091E3028093F10010928E
:1037A000F1008EEF8093E8006C960FB6F894DEBFC0
:1037B0000FBECDBFDF91CF91FF91EF91BF91AF9140
:1037C0009F918F917F916F915F914F913F912F9139
:1037D0001F910F91FF90EF90DF90CF900F900FBE51
:1037E0000F901F9018959EEF9093E800C7CF10920E
:1037F000F100D5CF913059F48111D3CF413051052B
:1038000081F68091E3028D7F8093E302CACF9330EB
:1038100049F48111C6CF4130510519F68091E30278
:103820008260F2CF953041F48091E80080FFFCCFB8
:1038300020682093E300B5CF963009F0A9C00B8D26
:103840001C8D22E01092E9001092E1021092E00239
:10385000F2122EC01092DF021092DE020E948E1130
:103860001F8299E09983FA8291E09E8390EA98877B
:103870009AEF99872091E0023091E102275F3F4F54
:103880003C832B838D831092E9001092E102109209
:10389000E0021093DF020093DE0249E050E0BE0137
:1038A0006F5F7F4F80E00E9468110E948E1179CF78
:1038B0001093DF020093DE020E947210DC01129668
:1038C0000D911C910115110509F451C1D801ED911B
:1038D000FC910480F581E02DBE016B5E7F4FC80135
:1038E0000995009709F03EC1F80100851185EACFDE
:1038F000F3E0FF120EC08F89882309F440C08230A4
:1039000061F440E860E18EE79BE10E94351181118E
:1039100048CF81E28093EB0047CF813029F440E823
:103920006BE082E79BE1F1CF833099F70E94721040
:10393000DC011296ED90FC908E010F5F1F4F680125
:10394000E114F10479F0D701ED91FC910680F78143
:10395000E02DB801C7010995080F111DF701E0849A
:10396000F184EECFD8011C92F60101900020E9F716
:103970003197BF016C197D0940E0C601C6CF6CE5E7
:103980007BE1FB01449150E080E80E94681109CF7F
:10399000973009F4BECF983021F481E08093F10094
:1039A00000CF993009F0FDCE837009F0B2CFEEE57B
:1039B000F1E081E031E096E32191222371F08093E0
:1039C000E9003093EB00DF0111972C912093EC007C
:1039D0009093ED008F5F873079F78EE78093EA0050
:1039E0001092EA008F898093F302DBCE8B8D9C8D41
:1039F0001092E9001092E1021092E0029093DF022F
:103A00008093DE02898D811192C08E899D89913AC1
:103A100049F4813209F07DCF47E050E067E071E082
:103A200080E0B3CF913209F074CF833269F48F898B
:103A3000988DB0E0A0E08093030190930401A093DF
:103A40000501B0930601ADCE803269F48091E800A3
:103A500082FFFCCF67E087E091E00E94BF118BEF0F
:103A60008093E8009ECE823209F09BCE8F898093AE
:103A70000E01EEEFFFE7859194918B3F9C4D51F144
:103A8000E0E0F8E08091070190910801A091090120
:103A9000B0910A01803B9440A105B105F1F48091F9
:103AA0000E0180FD1AC0EE3F8AE0F80789F587E72E
:103AB00097E791838083809160008093E20288E1A0
:103AC0009BE00FB6F894A895809360000FBE90938A
:103AD000600067CEEEEFFAE0D5CF80819181873725
:103AE000974709F05ECEA895809160008861809329
:103AF00060008091E20280936000EE3F2AE0F207CE
:103B000089F08091FE0A9091FF0A9183808349CECB
:103B1000808191818737980751F29093FF0A8093B3
:103B2000FE0AC5CF1092FF0A1092FE0A3ACE0E94FA
:103B30007210DC0112960D911C910115110509F40A
:103B4000E8CED801ED91FC910190F081E02DBE010D
:103B50006B5E7F4FC8010995811123CEF801008566
:103B60001185EBCF181619060CF41BCED2CEF1E05E
:103B7000FF12BECE60E67BE104CF1F920F920FB61C
:103B80000F9211242F933F938F939F93AF93BF93E3
:103B90008091630290916402A0916502B0916602E7
:103BA0003091920123E0230F2D3758F50196A11D86
:103BB000B11D209392018093630290936402A093BD
:103BC0006502B09366028091930190919401A09157
:103BD0009501B09196010196A11DB11D80939301AD
:103BE00090939401A0939501B0939601BF91AF91EA
:103BF0009F918F913F912F910F900FBE0F901F902B
:103C0000189526E8230F0296A11DB11DD2CF1F9251
:103C10000F920FB60F9211242F933F934F935F9300
:103C20006F937F938F939F93AF93BF93CF93DF93C4
:103C3000EF93FF9380918F01882389F08091F8069C
:103C400081110DC080918E01811109C090918D016B
:103C5000E0918B01F0918C01808189278083809194
:103C60008A01882309F49CC0809186019091870184
:103C7000A0918801B0918901892B8A2B8B2B09F4A3
:103C80008FC08091860190918701A0918801B091A9
:103C900089010197A109B109809386019093870159
:103CA000A0938801B0938901892B8A2B8B2B09F073
:103CB00077C0D1E0E0918401F0918501AF014F5FC1
:103CC0005F4F50938501409384012491822F807F20
:103CD000C22FCF70803821F48C2F0E942713EACF97
:103CE000803919F5E0914C07F0914D0709958D2722
:103CF00080938E01E0918401F0918501CF010196BE
:103D0000909385018093840164918091FB06C8178C
:103D100088F6C13021F4809183018111CBCF67FDFA
:103D2000C9CF8C2F0E94AA12C5CF87FD4CC03296F6
:103D3000F0938501E0938401FA014491A0919001F0
:103D4000B0919101322F242F0E942F336C507E4F5F
:103D50008F4F9F4F28EE33E040E050E00E940D333C
:103D60002093860130938701409388015093890105
:103D70008091860190918701A0918801B09189017D
:103D8000892B8A2B8B2B61F481E090E0A0E0B0E0DE
:103D90008093860190938701A0938801B093890155
:103DA000FF91EF91DF91CF91BF91AF919F918F9153
:103DB0007F916F915F914F913F912F910F900FBE27
:103DC0000F901F901895803E29F410928501109253
:103DD000840170CF803F09F06DCF10928A01E0CF4F
:103DE0001F920F920FB60F9211248F939F93AF9350
:103DF000BF93EF93FF938091FA06882309F454C090
:103E00008091F4069091F506A091F606B091F70620
:103E1000892B8A2B8B2BA1F190918201E09180015B
:103E2000F09181018081892780838091F4069091AF
:103E3000F506A091F606B091F706181619061A06AF
:103E40001B069CF48091F4069091F506A091F6066D
:103E5000B091F7060197A109B1098093F4069093F8
:103E6000F506A093F606B093F706FF91EF91BF9188
:103E7000AF919F918F910F900FBE0F901F9018954B
:103E80001092F8061092FA0680916F008D7F809351
:103E90006F0080918201E0918001F0918101908119
:103EA000809589238083E1CF80918E018111DDCFC0
:103EB00090918201E0918001F091810180818927B8
:103EC000F1CFECEFF6E01382128288EE93E0A0E0EF
:103ED000B0E084839583A683B78388E691E09183DD
:103EE00080838FEF9FEF9587848780EB80935D07BA
:103EF00080935C0780915B0720E3829FC0011124BF
:103F000090935A0780935907EEE4F7E08AE791E02F
:103F1000918380831582168280E1878314821382C5
:103F2000118683EF9DE090934D0780934C07089591
:103F3000789484B5826084BD84B5816084BD85B584
:103F4000826085BD85B5816085BD80916E00816090
:103F500080936E0010928100809181008260809336
:103F60008100809181008160809381008091800038
:103F700081608093800080919100826080939100A5
:103F80008091910081608093910080919000816088
:103F9000809390008091C10084608093C1008091E3
:103FA000C10082608093C1008091C10081608093D4
:103FB000C1008091C30081608093C3008091C000E4
:103FC00082608093C0008091C20081608093C200B3
:103FD00080917A00846080937A0080917A00826078
:103FE00080937A0080917A00816080937A0080913A
:103FF0007A00806880937A001092F3021092E302B4
:104000001092E5028091D70081608093D70080EA0A
:104010008093D80089B5806189BD89B5826089BDEA
:1040200009B400FEFDCF61E070E080E090E00E9406
:10403000F2118091D8008F7C80618093D8008091AC
:10404000E000807F8093E0008091E1008E7E80938D
:10405000E1008DE08093E200559A209A81EC8093F4
:104060007C0085B1806F85B984B1877E84B984B1C5
:10407000876E84B95E9A5F988AB1806D8AB9769AA4
:104080006E9881B3806F81BB899880B38D7080BB3F
:1040900080E58CBD81E08DBD85E090E00E94CF136E
:1040A0005F9A85E090E00E94CF135E985C98ECE008
:1040B000FBE084918EBD00000DB407FEFDCF31966C
:1040C0000BE0E931F007A9F75C9A81E8809364007E
:1040D000809165008160809365000E94D41382FF07
:1040E00046C02D980E94D41384788438D9F42D9A30
:1040F00088EC90E00E94CF132F9882E090E00E941D
:104100008E328F3F29F06FEF82E090E00E9496326E
:1041100084EF91E00E94CF132F9A0E94D4138478E9
:104120008438D9F30E94D41384718431D9F42D9A40
:1041300088EC90E00E94CF132E9882E090E00E94DD
:104140008E32882329F060E082E090E00E9496326F
:1041500084EF91E00E94CF132E9A0E94D4138471B1
:104160008431D9F388EC90E00E94CF13B6CF2D9A1A
:1041700082E090E00E948E32882309F48BC13E9A3F
:104180003F9A81E080939701809164008E7F8093B5
:10419000640080917A00806480937A0080917A0034
:1041A00086FDFCCFC0917800D09179000E94CD119E
:1041B000AB01BC01CE01B0E0A0E0DC01992788276B
:1041C0008C019D01040F151F261F371FC901B8015F
:1041D00020916400216020936400611571058105C0
:1041E000910511F00E94243180E18093550785E00C
:1041F0000E9452138DE00E945213CC24C394D12C00
:10420000C2E0AC2EB12CD3E08D2E912C15E0212EE6
:10421000312C84E38093690285E180936A021092D5
:104220006C0210926B02FCE3F093700296E19093A3
:104230007102D0927302C092720293E4909377025B
:1042400080937802B0927A02A092790297E49093D8
:104250007E0280937F02909281028092800246E2E9
:10426000409308028FE48093090210920B0210928F
:104270000A029AE390930F0221E520931002D09254
:104280001202C0921102809316028DE480931702ED
:10429000B0921902A092180256E650931D02209384
:1042A0001E02D0922002C0921F029BE7909324022C
:1042B00080932502B0922702A092260293E9909360
:1042C0002B0263E560932C0290922E0280922D02C5
:1042D0008FE88093320287E780933302A4E0B0E056
:1042E000B0933502A09334028FE780933902E2E85D
:1042F000E0933A0230923C0220923B027AE67093BD
:10430000400280934102C6E0D0E0D0934302C093C4
:10431000420232E530934702A1E8A093480230926E
:104320004A0220924902F0934E0280934F02D093AA
:104330005102C093500240935502E09356023092CE
:10434000580220925702EFE0E0935C0280935D02F6
:10435000D0935F02C0935E021092D0018CE58093EF
:10436000D1011092D3011092D2018DE08093D70138
:1043700085E68093D801D092DA01C092D9014093AA
:10438000DE018093DF01B092E101A092E0018BE3B6
:104390008093E5017093E6019092E8018092E70135
:1043A0006093EC0188E68093ED01B092EF01A0925A
:1043B000EE018093F30189E68093F4019092F60177
:1043C0008092F5018AE78093FA015093FB01B09245
:1043D000FD01A092FC019093010280E6809302020D
:1043E000E4E0F0E0F0930402E093030284E58093BC
:1043F000AD0189E28093AE011092B0011092AF013D
:104400003093B4018FE38093B501D092B701C0928D
:10441000B6013093BB018AE58093BC01D092BE0106
:10442000C092BD012093C20182E78093C301D09264
:10443000C501C092C401909398018AE080939901CC
:1044400096E890939F018093A00199E79093A6012D
:104450008093A7012FB7F894809163029091640232
:10446000A0916502B09166022FBF20915607F82FE8
:10447000F21B2F2FD0915707DD2389F0F0935807B7
:104480001092570780E090E0892B09F4C2CE0E9479
:104490000000B6CE109297013E983F9875CE3091AD
:1044A0005507F31740F42F5F231760F781E083BFB0
:1044B000889513BEE7CFC1E0C09357078093560796
:1044C00080915107909152070196909352078093E3
:1044D000510780E00E94161080910201882339F074
:1044E0008A3011F40C94AE2F0E940610CBCFE090CE
:1044F000DC02F090DD0287010F5F1F4F1093DD0299
:104500000093DC0280910101883209F440C608F072
:1045100008C1843109F439C608F0A3C0882309F41E
:10452000AAC18A3009F4DAC580910101833209F405
:1045300083C710F00C94682C843111F40C947B2DFB
:1045400010F00C94602C882311F40C94F62C8A3013
:1045500059F660905D07062C000C7708C091DA02CE
:104560000C2E000CDD0BB301675F7F4FEE24E3944C
:1045700000E920EA4AE750E1CE010E94DC13E09115
:104580008502EE0FFF0BE15EFE4F2081318187E057
:10459000829FF001839FF00D1124E759FD4F618147
:1045A000660D772D711D808148EF5FE08C0F9D2F88
:1045B000911D0E94C9130E94A9160E94EE158091B8
:1045C00068028F5F809368026BE00E94E133911173
:1045D0000CC080916702823040F444E150E060E01A
:1045E00070E088E49DE00E94F60D20916802822F21
:1045F0006EE10E94E133911105C0809167028F5FE7
:10460000809367028091670281110C94362D60912E
:104610005D07062E000C770B615C7F4F8091DA02FC
:10462000082E000C990BE12C05E125E148EE5EE037
:1046300088960E94DC1380916702863008F454CF7C
:1046400010926802109267028091C8028F5F809377
:10465000C802833010F40C94782D84E68093010115
:1046600043CF813209F4EAC5833209F47EC68E3124
:1046700009F05ACFC091DA026091DB02062E000CDD
:10468000770B6C1B7109C7FD7395072E000C880B07
:10469000990B0E9495312DEC3CEC4CEC5DE30E94B3
:1046A000D0312B013C016C2FCC0F770B880B990B71
:1046B0000E9495319B01AC01C301B2010E943F33BE
:1046C0000E94AB336093DA02C0915D0760915C0792
:1046D000062E000C770B6C1B7109C7FD7395072E16
:1046E000000C880B990B0E9495312DEC3CEC4CECA6
:1046F0005DE30E94D0312B013C016C2FCC0F770B76
:10470000880B990B0E9495319B01AC01C301B2014A
:104710000E943F330E94AB3360935D070E940817ED
:1047200003CF863409F420C788F5823309F4C2C662
:104730008C3309F0F9CEC80168E170E00E940334BF
:10474000892B99F4809190028F5F8093900248E2C8
:1047500050E060E070E084EC90E00E94F60D9091F3
:104760008F0281E0891B80938F02809190028530B7
:1047700008F4DACE109290028091C8028F5F809385
:10478000C802833008F4ECC684E6ECC58A3509F427
:10479000D7C7843611F40C94C12B803509F0C4CEF0
:1047A000C091DA026091DB02062E000C770B6C1BC5
:1047B0007109C7FD7395072E000C880B990B0E9499
:1047C00095312DEC3CEC4CE45EE30E94D0312B01A2
:1047D0003C016C2FCC0F770B880B990B0E94953105
:1047E0009B01AC01C301B2010E943F330E94AB3375
:1047F0006093DA02C0915D0760915C07062E000CA1
:10480000770B6C1B7109C7FD7395072E000C880B85
:10481000990B0E9495312DEC3CEC4CE45EE30E9438
:10482000D0312B013C016C2FCC0F770B880B990BEF
:104830000E9495319B01AC01C301B2010E943F333C
:104840000E94AB3360935D078091D6029091D702AE
:1048500003701127012B51F42091D4023091D5021D
:104860008217930708F051C70E94C5149093D7028E
:104870008093D60259CEC091DA026091DB02062EF7
:10488000000C770B6C1B7109C7FD7395072E000C8C
:10489000880B990B0E9495312DEC3CEC4CE45EE3C7
:1048A0000E94D0312B013C016C2FCC0F770B880B71
:1048B000990B0E9495319B01AC01C301B2010E948A
:1048C0003F330E94AB336093DA02C0915D07609181
:1048D0005C07062E000C770B6C1B7109C7FD7395E6
:1048E000072E000C880B990B0E9495312DEC3CECA7
:1048F0004CE45EE30E94D0312B013C016C2FCC0FC5
:10490000770B880B990B0E9495319B01AC01C30179
:10491000B2010E943F330E94AB3360935D078091E8
:10492000D6029091D7026AE070E00E94EF33CB018B
:104930006AE070E00E94EF33009719F024E02093C2
:104940005B078330910560F023E020935B0786309E
:10495000910530F0099709F46EC082E080935B07FF
:1049600080915B0700E3809FC001112490935A0758
:10497000809359070E9480150E9419170E940817FA
:1049800090910001E92FF0E08091D302682F70E050
:10499000C6E0CE9F9001CF9F300D1124D901A60F04
:1049A000B71FAA0FBB1FA35DBE4F4C914093D2020D
:1049B0003197CE9FA001CF9F500D1124FA01E60F31
:1049C000F71FEE0FFF1FE35DFE4F408140938A0209
:1049D000FB013197E20FF31FEE0FFF1FE35DFE4F68
:1049E0004081409389026F5F7F4F620F731FFB010D
:1049F000EE0FFF1FE35DFE4F20812093880292306F
:104A0000E1F4813011F00C94F82F2091BD022111B6
:104A100004C02091AF02222319F021E02093C702A5
:104A20002FEF20938B02923009F5811143C081E072
:104A30008093860244C081E091CF91110C941E3086
:104A4000833011F00C940B308091B502811104C0B9
:104A50008091A702882319F081E08093C50283E644
:104A600003C0811105C08BE080938B028FEFE0CFF4
:104A7000813011F48AE0F8CF823011F489E0F4CF6C
:104A8000833011F488E0F0CF843011F487E0ECCF6C
:104A9000853061F7C0938B02E9CF843011F483E055
:104AA000E3CF833011F482E0DFCF8230F9F69093C8
:104AB0008B02DCCF813009F02CC190938602C0912B
:104AC0008B02C33639F48091CA02882319F081E041
:104AD0008093D0024091D0020091DC021091DD025F
:104AE000C8016CE070E00E9403349C01442309F487
:104AF00073C0892B49F550915C07AFECB2E08AECAA
:104B000092E0FD0162917C91DF017083618360918D
:104B1000CE02611140E01092CF026091CA02611191
:104B200009C16091CB02611105C16091CC02611194
:104B300003C16091CD026111FFC08E179F0709F775
:104B40004093D00250935C078091B502811104C05C
:104B50008091A702882381F08091CB02882361F0A5
:104B60008091D6029091D70203969093D5028093BC
:104B7000D40280E5809301018091A002811104C0DC
:104B800080919702882381F08091CC02882361F084
:104B90008091D6029091D70206969093D502809389
:104BA000D40280E5809301018091BC02811104C090
:104BB0008091AE02882381F08091CD02882361F03C
:104BC0008091D6029091D70209969093D502809356
:104BD000D40280E5809301018091870290910101C8
:104BE000EFEBF2E04C2F50E06081662361F0BF01F3
:104BF000635B72406417750731F42115310519F4B0
:104C0000811101C09CE3319763EB72E06E177F075F
:104C100059F7E1EBF2E04C2F50E06081662361F040
:104C2000BF01655A72404617570731F42115310507
:104C300019F4813009F49CE33197A5EAB2E0AE178C
:104C4000BF0759F74091860250E0E2EAF2E06CE9D2
:104C500072E0A081AA2361F0DF01AC59B2404A178B
:104C60005B0731F42115310519F4823009F49CE316
:104C700031976E177F0769F7E9E9F2E063E972E0BF
:104C8000A081AA2361F0DF01A359B2404A175B0754
:104C900031F42115310519F4833009F49CE331977F
:104CA0006E177F0769F7909301010E942E1780937A
:104CB000C9022091D302243029F4D1E0909100015F
:104CC0009111D0E090918C02891709F4ACC0883022
:104CD00009F078C1809100018330E9F58C2F90E0D4
:104CE000FC01ED54FD4F3081311106C0FC01EB5544
:104CF000FD4F3081332311F121502093D302015015
:104D000011091093DD020093DC028CE38093010112
:104D100022C0823011F483E08BCE833011F484E022
:104D200087CE843011F485E083CE853009F0C7CE7C
:104D300086E07ECE57EEF9CE50EBFFCE0197FC0118
:104D4000ED54FD4F20812111DACF8B559D4FFC0191
:104D500080818111D4CF8091C9028430E9F480919F
:104D6000D3028823C9F0909189022FEF290F2330B5
:104D700010F0953089F49091D202923069F0D111FF
:104D80000BC081508093D30242E150E060E070E0BC
:104D900088EB91E00E94F60D8091C9028830C1F441
:104DA0008091D3028530A0F4909188029150943084
:104DB00078F49091D202923059F08F5F8093D302B1
:104DC00042E150E060E070E088EB91E00E94F60D77
:104DD0008091C9028031A1F480918A028250823090
:104DE00078F480910001882359F08150809300016C
:104DF00042E150E060E070E088EB91E00E94F60D47
:104E00008091C902843111F0803259F49091D3021B
:104E1000923039F490910001913019F494E190931B
:104E2000010180938C028091D202823009F095C0FA
:104E300080918D0290918E02019690938E028093C4
:104E40008D0260E370E00E940334892B09F085C075
:104E5000809100018F5F8093000110928E0210926A
:104E60008D028091C7028823D9F08091BD02811103
:104E700017C08091AF02811113C08091D60290912A
:104E8000D70201969093D7028093D60244E150E076
:104E900060E070E080EE96E00E94F60D1092C7028E
:104EA0008091C6028823D9F08091BA02811117C07F
:104EB0008091AC02811113C08091D6029091D702EB
:104EC00001969093D7028093D60244E150E060E0CF
:104ED00070E080EE96E00E94F60D1092C60280917E
:104EE000C5028823D9F08091B502811117C0809145
:104EF000A702811113C08091D6029091D70201962A
:104F00009093D7028093D60244E150E060E070E0D5
:104F100080EE96E00E94F60D1092C5028091C402C8
:104F20008823D9F08091B402811117C08091A60224
:104F3000811113C08091D6029091D702019690936F
:104F4000D7028093D60244E150E060E070E080EE4A
:104F500096E00E94F60D1092C4028091C2029091D8
:104F6000C30201969093C3028093C2022091590715
:104F700030915A072817390708F0D6CA8091DC0209
:104F80009091DD0268E170E00E940334892B09F002
:104F9000CBCA1092C3021092C2020E94793064E020
:104FA00070E00E940334009709F06BC08091B30257
:104FB0008111F3CF8091B4028111EFCF81E0809312
:104FC000B302B2CA843009F047C080910001813039
:104FD00009F0C1CE8C2F90E0FC01ED54FD4F3081E3
:104FE000311106C0FC01EB55FD4F3081332329F10F
:104FF0002F5F2093D302015011091093DD0200931B
:10500000DC028CE3809301018091C902823009F0B7
:10501000A2CE8091D2028350823008F09CCE809143
:1050200000018F5F8093000142E150E060E070E09A
:1050300088EB91E00E94F60D8ECE0197FC01ED54B5
:10504000FD4F20812111D7CF8B559D4FDC018C91D5
:10505000882309F480CECFCF8130B1F680918A02C7
:10506000843009F078CE8091000181508093000156
:1050700042E150E060E070E088EB91E00E94F60DC4
:10508000C3CF8130910561F48091A502811185CF54
:105090008091A602811181CF81E08093A50244CA4C
:1050A0008230910561F480919C02811176CF8091CC
:1050B0009D02811172CF81E080939C0235CA0397D3
:1050C00009F06BCF80919302811167CF8091940298
:1050D000811163CF81E08093930226CAC091DA02E6
:1050E0006091DB02062E000C770B6C1B7109C7FD6B
:1050F0007395072E000C880B990B0E9495312DECAF
:105100003CEC4CE45EE30E94D0312B013C016C2F5F
:10511000CC0F770B880B990B0E9495319B01AC014A
:10512000C301B2010E943F330E94AB336093DA02A5
:10513000C0915D0760915C07062E000C770B6C1B1D
:105140007109C7FD7395072E000C880B990B0E94FF
:1051500095312DEC3CEC4CE45EE30E94D0312B0108
:105160003C016C2FCC0F770B880B990B0E9495316B
:105170009B01AC01C301B2010E943F330E94AB33DB
:1051800060935D070E941917CFC90E948015C091D6
:10519000DA026091DB02062E000C770B6C1B7109A2
:1051A000C7FD7395072E000C880B990B0E94953153
:1051B0002DEC3CEC4CEC5EE30E94D0312B013C0129
:1051C0006C2FCC0F770B880B990B0E9495319B01AC
:1051D000AC01C301B2010E943F330E94AB33609324
:1051E000DA02C0915D0760915C07062E000C770B18
:1051F0006C1B7109C7FD7395072E000C880B990B6A
:105200000E9495312DEC3CEC4CEC5EE30E94D031D9
:105210002B013C016C2FCC0F770B880B990B0E9454
:1052200095319B01AC01C301B2010E943F330E9442
:10523000AB3360935D070E94191770CAC091DA0200
:105240006091DB02062E000C770B6C1B7109C7FD09
:105250007395072E000C880B990B0E9495312DEC4D
:105260003CEC4CEC5DE30E94D0312B013C016C2FF7
:10527000CC0F770B880B990B0E9495319B01AC01E9
:10528000C301B2010E943F330E94AB336093DA0244
:10529000C0915D0760915C07062E000C770B6C1BBC
:1052A0007109C7FD7395072E000C880B990B0E949E
:1052B00095312DEC3CEC4CEC5DE30E94D0312B01A0
:1052C0003C016C2FCC0F770B880B990B0E9495310A
:1052D0009B01AC01C301B2010E943F330E94AB337A
:1052E00060935D070E9408178091D9029091D802BF
:1052F000890F893258F58093D902C0915D070C2E31
:10530000000CDD0B6090DA02062C000C7708BE0161
:10531000675F7F4FEE24E39400E920EA4AE750E11B
:10532000C3010E94DC13BE01655F7F4FE12C02E2E6
:1053300029E14BE75FE0C30180960E94DC130E94E5
:10534000D8140E94EE150E94A916CEC81092D90258
:105350008091D6029091D70205969093D5028093C2
:10536000D40286E480930101DFC8C091DA02609123
:10537000DB02062E000C770B6C1B7109C7FD7395C1
:10538000072E000C880B990B0E9495312DEC3CECFC
:105390004CEC5DE30E94D0312B013C016C2FCC0F13
:1053A000770B880B990B0E9495319B01AC01C301CF
:1053B000B2010E943F330E94AB336093DA02C09186
:1053C0005D0760915C07062E000C770B6C1B710962
:1053D000C7FD7395072E000C880B990B0E94953121
:1053E0002DEC3CEC4CEC5DE30E94D0312B013C01F8
:1053F0006C2FCC0F770B880B990B0E9495319B017A
:10540000AC01C301B2010E943F330E94AB336093F1
:105410005D073701B2E06B0E711C7092DD02609285
:10542000DC020E9408178091D9029091D802890F5E
:105430008136C0F58093D90260905D07062C000C80
:105440007708C091DA020C2E000CDD0BB301675F08
:105450007F4FEE24E39400E920EA4AE750E1CE01D1
:105460000E94DC13B301655F7F4FE12C02E229E16A
:105470004BE75FE0CE0180960E94DC130E94D814B7
:105480000E94EE15B301645F7F4FCE01019620911B
:10549000D80221110EC405E226E240EB5CE00E9436
:1054A000DC1322C81092D9028091D6029091D702C3
:1054B0000F9653CFC091DA026091DB02062E000CEA
:1054C000770B6C1B7109C7FD7395072E000C880BB9
:1054D000990B0E9495312DEC3CEC4CEC5EE30E9464
:1054E000D0312B013C016C2FCC0F770B880B990B23
:1054F0000E9495319B01AC01C301B2010E943F3370
:105500000E94AB336093DA02C0915D0760915C0743
:10551000062E000C770B6C1B7109C7FD7395072EC7
:10552000000C880B990B0E9495312DEC3CEC4CEC57
:105530005EE30E94D0312B013C016C2FCC0F770B26
:10554000880B990B0E9495319B01AC01C301B201FC
:105550000E943F330E94AB3360935D070C9494220A
:1055600010928F028AE5FECEC091DA026091DB02D2
:10557000062E000C770B6C1B7109C7FD7395072E67
:10558000000C880B990B0E9495312DEC3CEC4CE4FF
:105590005EE30E94D0312B013C016C2FCC0F770BC6
:1055A000880B990B0E9495319B01AC01C301B2019C
:1055B0000E943F330E94AB336093DA02C0915D07D3
:1055C00060915C07062E000C770B6C1B7109C7FD00
:1055D0007395072E000C880B990B0E9495312DECCA
:1055E0003CEC4CE45EE30E94D0312B013C016C2F7B
:1055F000CC0F770B880B990B0E9495319B01AC0166
:10560000C301B2010E943F330E94AB3360935D0738
:1056100087EF80935C078EED8093DB02809192028E
:10562000882361F1813011F00C9494228091D6028C
:105630009091D70203701127012B49F42091D402D5
:105640003091D5028217930710F40E94C5149093ED
:10565000D7028093D6022091D4023091D502281728
:10566000390711F00C94942268E770E080E090E034
:105670000E94F2111092920282E374CE8091D602BF
:105680009091D70203701127012B49F42091D40285
:105690003091D5028217930710F40E94C51490939D
:1056A000D7028093D6022091D4023091D5022817D8
:1056B000390711F00C94942221E02093920230914A
:1056C000D1022FE0231B209391023091C10234308C
:1056D00029F4220F209391021092C102209191028D
:1056E00027FD1092910220919102820F911D27FDBA
:1056F0009A959093D5028093D40268E770E080E099
:1057000090E00E94F2110C9494222091CB0222236B
:1057100021F01092B5021092A7022091CC02222310
:1057200021F01092A002109297022091CD02222324
:1057300021F01092BC021092AE021092010196C8A4
:105740001092D30283E080930001C093D2021092A2
:10575000BF021092BE021092BD021092B1021092CE
:10576000B0021092AF02D092DD02C092DC02109221
:10577000D1021092D002C093CA02109201010C947F
:10578000942287EF80935C078EED8093DB02C091BB
:10579000DA026EED7FEF6C1B7109C7FD7395072E62
:1057A000000C880B990B0E9495312DEC3CEC4CE4DD
:1057B0005EE30E94D0312B013C016C2FCC0F770BA4
:1057C000880B990B0E9495319B01AC01C301B2017A
:1057D0000E943F330E94AB336093DA02C0915D07B1
:1057E00067EF7FEF6C1B7109C7FD7395072E000CE7
:1057F000880B990B0E9495312DEC3CEC4CE45EE358
:105800000E94D0312B013C016C2FCC0F770B880B01
:10581000990B0E9495319B01AC01C301B2010E941A
:105820003F330E94AB3360935D070E9419170E94BB
:105830002E178093C902803209F05DC31092C8020E
:105840001092C9021092DD021092DC021092D30273
:1058500083E08093000181E08093D2021092C7021E
:105860001092C6021092C5021092C4021092C30296
:105870001092C2021092D8021092C10287E0809367
:105880005B07E3EBF2E025EA32E08CE992E063E9C2
:1058900072E0AAECB2E01192E90119929E01EC01CA
:1058A0001992CE01EB011992BE011D92D2E0E23CA9
:1058B000FD0789F781E08093B3028093CA0252CE3C
:1058C0008E3109F487C1813209F417CD0C9474220A
:1058D0008C3309F495C208F068C0883209F4EFC12E
:1058E000823311F00C947422C0915D070C2E000CD1
:1058F000DD0B6090DA02062C000C7708BE01675FB2
:105900007F4FEE24E39400E920EA4AE750E1C30127
:105910000E94DC13E0918502EE0FFF0BE15EFE4F6B
:105920002081318187E0829FF001839FF00D112457
:10593000E759FD4F61816C0F7D2F711D808148EF0C
:105940005FE0860D972D911D0E94C913809168021A
:105950008F5F8093680268E20E94E133911105C075
:10596000809167028F5F80936702BE01625D7F4F07
:10597000E12C0EE125E147E25FE0C30182960E943F
:10598000DC131092DB0283ED80935C078091670249
:10599000823038F010926802109267028AE5809394
:1059A00001010E94D8140C947422803509F46AC253
:1059B000843609F4A0C2863411F00C9474226091EC
:1059C0005D07062E000C770B675F7F4F8091DA0230
:1059D000EE24E39400E920EA4AE750E1082E000CA7
:1059E000990B0E94DC130E94071A59C160905D0751
:1059F000062C000C7708C091DA020C2E000CDD0B8F
:105A0000B301675F7F4FEE24E39400E920EA4AE7A1
:105A100050E1CE010E94DC13E0918502EE0FFF0BF6
:105A2000E15EFE4F2081318187E0829FF001839FFC
:105A3000F00D1124E759FD4F6181660D772D711D21
:105A4000808148EF5FE08C0F9D2F911D0E94C9134C
:105A50000E94A9160E949B170E94D8140E94EE155E
:105A60000E9493190E94071A0C9474228130C9F481
:105A70001092DB028FEB80935C0760915D07062E2E
:105A8000000C770B625B7F4F8091DA02082E000CCE
:105A9000990BE12C0EE12CE148E75EE00D960C94A9
:105AA000192320FD0AC0823041F444E150E060E057
:105AB00070E084EC90E00E94F60D60915D07062E88
:105AC000000C770B65597F4F8091DA02082E000C8D
:105AD000990BE12C00E223E14CE25EE003960E9488
:105AE000DC131092DB0280EB80935C070C941B2389
:105AF0008AE50C942E23C0915D070C2E000CDD0B63
:105B00006090DA02062C000C7708BE01675F7F4FB9
:105B1000EE24E39400E920EA4AE750E1C3010E9441
:105B2000DC1310918502E12FEE0FFF0BE15EFE4FBB
:105B30002081318187E0829FF001839FF00D112445
:105B4000E759FD4F61816C0F7D2F711D808148EFFA
:105B50005FE0860D972D911D0E94C9130E94A91622
:105B6000809168028F5F809368026FE00E94E1334A
:105B7000911105C0809167028F5F809367028091C9
:105B8000670281110FC0BE01645D7F4FE12C0BE104
:105B900024E143EE5BE0C301CB960E94DC130E943C
:105BA000D8147DC0813059F4BE01615E7F4FE12C75
:105BB0000CE224E14BE65BE0C301C696EECF109207
:105BC0006802109267028EE1133009F088E2809338
:105BD0000101E5CFC0915D070C2E000CDD0B60903C
:105BE000DA02062C000C7708BE01675F7F4FEE24B7
:105BF000E39400E920EA4AE750E1C3010E94DC1384
:105C00000E94D8148091DC029091DD02019690935D
:105C1000DD028093DC02809168028F5F80936802CE
:105C200068E20E94E133911105C0809167028F5FA5
:105C3000809367021091670211110CC0E12C02E2FF
:105C400029E143E35CE0BE01655F7F4FC3018096BD
:105C50000E94DC131092DB0287EF80935C07112314
:105C6000E1F0BE01655F7F4FE12C02E229E14BE7E5
:105C70005FE0C30180960E94DC13123070F08091C7
:105C8000C1028F5F8093C102843069F41092DD02FB
:105C90001092DC0283E2809301010E94A9160E9407
:105CA000EE150C947422109268021092670281E241
:105CB000F2CFE12C05E226E24EE65DE0F0CBC091AA
:105CC0005D070C2E000CDD0B6090DA02062C000C38
:105CD0007708BE01675F7F4FEE24E39400E920EA76
:105CE0004AE750E1C3010E94DC13E0918502EE0F08
:105CF000FF0BE15EFE4F2081318187E0829FF00142
:105D0000839FF00D1124E759FD4F61816C0F7D2FAA
:105D1000711D808148EF5FE0860D972D911D0E94D7
:105D2000C913209168022F5F20936802822F6FE0D1
:105D30000E94E133911105C0809167028F5F8093CB
:105D4000670280916702811121C0BE016E5C7F4FA6
:105D5000E12C05E125E148EE5EE0C3018E960E944C
:105D6000DC1380916702863070F010926802109206
:105D700067028091C8028F5F8093C8028330F0F180
:105D800084E6809301010E94A91609CF813091F425
:105D9000BE01625B7F4FE12C0EE12CE148E75EE043
:105DA000C3010D960E94DC131092DB0289EC8093F4
:105DB0005C07D7CF20FD0AC0843040F444E150E0B6
:105DC00060E070E084EC90E00E94F60D60915D0769
:105DD000062E000C770B65597F4F8091DA02082E52
:105DE000000C990BE12C00E223E14CE25EE003960B
:105DF0000E94DC131092DB0280EBD9CF8AE5C1CF81
:105E000060905D07062C000C7708C091DA020C2E1A
:105E1000000CDD0BB301675F7F4FEE24E39400E9D4
:105E200020EA4AE750E1CE010E94DC13E0918502AE
:105E3000EE0FFF0BE15EFE4F2081318187E0829FF4
:105E4000F001839FF00D1124E759FD4F6181660D2C
:105E5000772D711D808148EF5FE08C0F9D2F911D84
:105E60000E94C91380918F02813011F40E949B1708
:105E70000E94D8140E94A9160E94EE150E94931940
:105E80000C94742260905D07062C000C7708C0917A
:105E9000DA020C2E000CDD0BB301675F7F4FEE249E
:105EA000E39400E920EA4AE750E1CE010E94DC13C6
:105EB000E0918502EE0FFF0BE15EFE4F2081318104
:105EC00087E0829FF001839FF00D1124E759FD4F79
:105ED0006181660D772D711D808148EF5FE08C0F29
:105EE0009D2F911D0E94C9130E949B170E94D814D8
:105EF0000E949319D4CE60905D07062C000C7708A1
:105F0000C091DA020C2E000CDD0BB301675F7F4FEE
:105F1000EE24E39400E920EA4AE750E1CE010E9432
:105F2000DC13E0918502EE0FFF0BE15EFE4F208156
:105F3000318187E0829FF001839FF00D1124E759A2
:105F4000FD4F6181660D772D711D808148EF5FE007
:105F50008C0F9D2F911D0E94C91380CD81E00E945E
:105F6000161002E020E043E45BE068E170E086E3C5
:105F700090E00E944B0E0E94061044E650E060E064
:105F800070E08DE298E00E94F60D68E270E080E03B
:105F900090E00E94F21144E650E060E070E08DE491
:105FA0009AE00E94F60D6CE172E080E090E00E94C1
:105FB000F2116CED75E080E090E00E94F21120E0BB
:105FC00049E15BE06AE270E08CE290E00E944B0EF7
:105FD0000E9406100E9477190E94771968EB7BE0F7
:105FE00080E090E00E94F211109202010C94742261
:105FF000843011F00C9410252091BA02211106C0B2
:106000002091AC02222311F40C94102521E020935E
:10601000C6020C941025823011F00C9410252091AA
:10602000B402211106C02091A602222311F40C947F
:10603000102521E02093C4020C941025933011F414
:106040000C943125913011F00C941025853011F00D
:106050000C944D2584E00C9434258F929F92AF923E
:10606000BF92CF92DF92EF92FF92CF93DF93EC013A
:10607000688179818A819B8161157105810591050E
:1060800021F464E279ED8BE597E02DE133EF41E017
:1060900050E00E94A43249015A019B01AC01A7EAD9
:1060A000B1E40E94C3326B017C01ACEEB4EFA501F8
:1060B00094010E94D132DC01CB018C0D9D1DAE1DDF
:1060C000BF1DB7FF03C00197A109B048888399831A
:1060D000AA83BB839F77DF91CF91FF90EF90DF90F2
:1060E000CF90BF90AF909F908F9008950E942D30D9
:1060F00008958FE091E00E942D300895B0E0A0E077
:1061000080930F0190931001A0931101B09312019D
:1061100008958F929F92AF92BF92CF92DF92EF92AB
:10612000FF92CF93DF93EC01688179818A819B8113
:10613000611571058105910521F464E279ED8BE526
:1061400097E02DE133EF41E050E00E94A432490195
:106150005A019B01AC01A7EAB1E40E94C3326B0172
:106160007C01ACEEB4EFA50194010E94D132C60EC1
:10617000D71EE81EF91EF7FE06C081E0C81AD10836
:10618000E10880E8F80AC882D982EA82FB82C70166
:10619000B6019F77DF91CF91FF90EF90DF90CF9086
:1061A000BF90AF909F908F9008958F929F92AF92E3
:1061B000BF92CF92DF92EF92FF92609113017091A4
:1061C00014018091150190911601611571058105E9
:1061D000910521F464E279ED8BE597E02DE133EF51
:1061E00041E050E00E94A43249015A019B01AC01F8
:1061F000A7EAB1E40E94C3326B017C01ACEEB4EFBC
:10620000A50194010E94D132C60ED71EE81EF91EC8
:10621000F7FE06C081E0C81AD108E10880E8F80A54
:10622000C0921301D0921401E0921501F092160170
:10623000C701B6019F77FF90EF90DF90CF90BF909E
:10624000AF909F908F900895609313017093140105
:10625000809315019093160108951F93FC019927CF
:106260008827BC01E89411911032E9F3193010F03D
:106270001E30C8F31B3251F01D3249F4689406C039
:106280000E945431610F711D811D911D1191105398
:106290001A30B0F33EF490958095709561957F4FDC
:1062A0008F4F9F4F1F910895592F482F372F262F1B
:1062B000660F771F881F991F660F771F881F991F0A
:1062C000620F731F841F951F660F771F881F991F0A
:1062D0000895BB27FB015527AA27880F991FAA1FDE
:1062E000A41710F0A41B83955051B9F7A05DAA33F1
:1062F00008F0A95DA193009779F7B111B1931192BC
:10630000CB010C948331DC01FC01672F7191772361
:10631000E1F7329704C07C916D9370836291AE1760
:10632000BF07C8F30895E89409C097FB3EF4909521
:106330008095709561957F4F8F4F9F4F9923A9F05E
:10634000F92F96E9BB279395F695879577956795ED
:10635000B795F111F8CFFAF4BB0F11F460FF1BC031
:106360006F5F7F4F8F4F9F4F16C0882311F096E9C4
:1063700011C0772321F09EE8872F762F05C0662372
:1063800071F096E8862F70E060E02AF09A95660F2B
:10639000771F881FDAF7880F9695879597F90895E4
:1063A0000E94E3310C9454320E94463238F00E942D
:1063B0004D3220F0952311F00C943D320C94433271
:1063C00011240C9488320E94653270F3959FC1F3BA
:1063D000950F50E0551F629FF001729FBB27F00D93
:1063E000B11D639FAA27F00DB11DAA1F649F6627E8
:1063F000B00DA11D661F829F2227B00DA11D621F37
:10640000739FB00DA11D621F839FA00D611D221FF0
:10641000749F3327A00D611D231F849F600D211DD4
:10642000822F762F6A2F11249F5750409AF0F1F057
:1064300088234AF0EE0FFF1FBB1F661F771F881FC0
:1064400091505040A9F79E3F510580F00C943D3289
:106450000C9488325F3FE4F3983ED4F386957795A9
:106460006795B795F795E7959F5FC1F7FE2B880F66
:10647000911D9695879597F9089597F99F6780E8FC
:1064800070E060E008959FEF80EC089500240A9486
:106490001616170618060906089500240A941216FF
:1064A0001306140605060895092E0394000C11F432
:1064B000882352F0BB0F40F4BF2B11F460FF04C0DF
:1064C0006F5F7F4F8F4F9F4F089557FD9058440F38
:1064D000551F59F05F3F71F04795880F97FB991F43
:1064E00061F09F3F79F08795089512161306140600
:1064F000551FF2CF4695F1DF08C01616170618068D
:10650000991FF1CF86957105610508940895E89467
:10651000BB2766277727CB0197F90895F999FECF16
:1065200092BD81BDF89A992780B50895262FF999D3
:10653000FECF1FBA92BD81BD20BD0FB6F894FA9A66
:10654000F99A0FBE01960895052E97FB1EF400944C
:106550000E94BB3257FD07D00E940D3307FC03D0C9
:106560004EF40C94BB3250954095309521953F4F99
:106570004F4F5F4F089590958095709561957F4F2F
:106580008F4F9F4F08950E942F33A59F900DB49F6A
:10659000900DA49F800D911D11240895B7FF0C94B8
:1065A000C3320E94C332821B930B08952F923F92F5
:1065B0004F925F926F927F928F929F92AF92BF9213
:1065C000CF92DF92EF92FF920F931F93CF93DF93BF
:1065D000CDB7DEB7CA1BDB0B0FB6F894DEBF0FBE1C
:1065E000CDBF09942A88398848885F846E847D8469
:1065F0008C849B84AA84B984C884DF80EE80FD806B
:106600000C811B81AA81B981CE0FD11D0FB6F894E0
:10661000DEBF0FBECDBFED010895A1E21A2EAA1B69
:10662000BB1BFD010DC0AA1FBB1FEE1FFF1FA21742
:10663000B307E407F50720F0A21BB30BE40BF50B3F
:10664000661F771F881F991F1A9469F760957095C8
:10665000809590959B01AC01BD01CF010895A29F4B
:10666000B001B39FC001A39F700D811D1124911D26
:10667000B29F700D811D1124911D08955058BB27A4
:10668000AA270E9456330C9454320E94463238F0A6
:106690000E944D3220F039F49F3F19F426F40C94F7
:1066A00043320EF4E095E7FB0C943D32E92F0E9453
:1066B000653258F3BA17620773078407950720F00D
:1066C00079F4A6F50C9487320EF4E0950B2EBA2FD0
:1066D000A02D0B01B90190010C01CA01A0011124E8
:1066E000FF27591B99F0593F50F4503E68F11A1694
:1066F000F040A22F232F342F4427585FF3CF469525
:1067000037952795A795F0405395C9F77EF41F1646
:10671000BA0B620B730B840BBAF09150A1F0FF0F10
:10672000BB1F661F771F881FC2F70EC0BA0F621FFC
:10673000731F841F48F4879577956795B795F795EC
:106740009E3F08F0B0CF9395880F08F09927EE0F81
:106750009795879508950E94B2336894B1110C946F
:10676000883208950E946D3288F09F5798F0B92FB3
:106770009927B751B0F0E1F0660F771F881F991F76
:106780001AF0BA95C9F714C0B13091F00E9487325F
:10679000B1E008950C948732672F782F8827B85F6F
:1067A00039F0B93FCCF3869577956795B395D9F7CE
:1067B0003EF490958095709561957F4F8F4F9F4FD8
:1067C000089587FB082E062687FD819567FD619554
:1067D0000E9417340EF4919507FC81950895AA1B29
:1067E000BB1B51E107C0AA1FBB1FA617B70710F0BC
:1067F000A61BB70B881F991F5A95A9F780959095EE
:10680000BC01CD01089597FB072E16F4009407D024
:1068100077FD09D00E94EF3307FC05D03EF4909538
:1068200081959F4F0895709561957F4F0895991BAD
:1068300079E004C0991F961708F0961B881F7A9577
:10684000C9F780950895EE0FFF1F0590F491E02D94
:1068500009940F931F93CF93DF938230910510F427
:1068600082E090E0E0916007F091610730E020E085
:10687000B0E0A0E0309799F42115310509F44AC041
:10688000281B390B24303105D8F58A819B8161158D
:10689000710589F1FB0193838283FE0111C0408160
:1068A00051810281138148175907E0F048175907B1
:1068B00099F4109761F012960C93129713961C930B
:1068C0003296CF01DF91CF911F910F9108950093E0
:1068D000600710936107F4CF2115310551F042177D
:1068E000530738F0A901DB019A01BD01DF01F8016E
:1068F000C1CFEF01F9CF9093610780936007CDCFAF
:10690000FE01E20FF31F81939193225031093983E5
:106910002883D7CF20915E0730915F07232B41F466
:106920002091190130911A0130935F0720935E077F
:1069300020911701309118012115310541F42DB72F
:106940003EB740911B0150911C01241B350BE09177
:106950005E07F0915F07E217F307A0F42E1B3F0BD1
:106960002817390778F0AC014E5F5F4F24173507C1
:1069700048F04E0F5F1F50935F0740935E0781936F
:1069800091939FCFF0E0E0E09CCFCF93DF9300970F
:10699000E9F0FC01329713821282A0916007B09156
:1069A0006107ED0130E020E01097A1F420813181F2
:1069B000820F931F20915E0730915F0728173907D8
:1069C00009F061C0F0935F07E0935E07DF91CF911C
:1069D0000895EA01CE17DF07E8F54A815B819E0141
:1069E00041155105B1F7E901FB83EA8349915991BA
:1069F000C40FD51FEC17FD0761F4808191810296C9
:106A0000840F951FE90199838883828193819B83F9
:106A10008A83F0E0E0E012968D919C9113970097A5
:106A2000B9F52D913C911197CD010296820F931FDC
:106A300020915E0730915F072817390739F63097A4
:106A400051F51092610710926007B0935F07A09311
:106A50005E07BCCFD383C28340815181840F951FD1
:106A6000C817D90761F44E5F5F4F88819981480F3D
:106A7000591F518340838A819B819383828321158F
:106A8000310509F0B0CFF0936107E09360079ECF26
:106A9000FD01DC01C0CF13821282D7CFB0E0A0E0AD
:106AA000E4E5F5E30C94D8328C01009751F4CB0166
:106AB0000E9429348C01C801CDB7DEB7E0E10C9407
:106AC000F432FC01E60FF71F9C0122503109E21756
:106AD000F30708F49DC0D901CD91DC911197C61739
:106AE000D70798F0C530D10530F3CE01049786174B
:106AF000970708F3C61BD70B2297C193D1936D93C9
:106B00007C93CF010E94C534D6CF5B01AC1ABD0A7D
:106B10004C018C0E9D1EA0916007B0916107512C15
:106B2000412CF12CE12C109731F580915E0790916A
:106B30005F078815990509F05CC04616570608F0EE
:106B400058C08091170190911801009741F48DB7BA
:106B50009EB740911B0150911C01841B950BE817B7
:106B6000F90708F055C0F0935F07E0935E07F9015D
:106B700071836083A0CF8D919C91119712966C9038
:106B8000129713967C901397A815B90559F56C01C7
:106B900042E0C40ED11CCA14DB0420F1AC014A1936
:106BA0005B09DA011296159780F062827382518335
:106BB0004083D9016D937C93E114F10471F0D70106
:106BC0001396FC93EE93129776CF22968C0F9D1F0F
:106BD000F90191838083F301EFCFF0936107E09394
:106BE000600769CF4816590608F42C017D01D301CE
:106BF0009ACFCB010E9429347C01009749F0AE0165
:106C0000B8010E940B36C8010E94C534870153CFDA
:106C100010E000E050CFFB01DC0102C001900D92BA
:106C200041505040D8F70895FB01DC0101900D92CE
:0A6C30000020E1F70895F894FFCF6B
:106C3A0003640AFFFFFFFF00E100000000000001FB
:106C4A000000000100000000006207800003010349
:106C5A000002000100000001000200030000000021
:106C6A00000200020003000000000005000100010C
:106C7A0000010004000300020003000300020003F5
:106C8A000001000100010001000100010000C180B3
:106C9A00810000000000000086102512A7109C1039
:0E6CAA00ED10AB10C91000000000C414000073
:00000001FF
